:10000000F01F0010A5540000A3540000A3540000EA
:10001000A3540000A3540000A354000000000000FB
:10002000000000000000000000000000A3540000D9
:10003000A354000000000000A3540000CD240000E1
:10004000D5220000D5220000D5220000D5220000D4
:10005000D5220000D5220000D5220000D5220000C4
:10006000D5220000D5220000D5220000D5220000B4
:10007000D5220000A1540000A1540000C1000000DE
:100080006D2500008525000099270000B12700009C
:10009000A1540000F5280000A1540000A154000064
:1000A000A1540000A1540000A1540000A15400007C
:1000B000A1540000A1540000A1540000A15400006C
:1000C000554B10B51A6801321A60544B1A68544BDC
:1000D000D2B2302A69D01ADC182A44D012DC082A9D
:1000E00032D0102A00D094E04E4A002111604E49CF
:1000F0000A68501C08604D49895C4D4AC9B21160BC
:10010000282287E0202A63D0282A32D081E0482A9A
:100110005ED004DC382A51D0402A53D079E0502AEE
:1001200060D0582A75D13F490A68501C0860404980
:1001300008684049C0B288543F4A0221FF3111602B
:1001400080221021D20563E0374A00211160116836
:10015000481C1060354A515C354AC9B211602822EA
:100160001A6001223CE030490A68501C08602F499F
:1001700009E02D4A314910680968884207D21168A0
:10018000481C1060294A515C294AC9B240E02C4AF7
:1001900011688022D205002901D0202138E02649AB
:1001A0000220FF300860102132E08022D2051021A9
:1001B000116008221A608122520011E08221490058
:1001C0001D4A25E01E4A1168042201291AD11DE0AA
:1001D0008022D2051021116008221A600422FF3209
:1001E000154B17E00F4A1168481C1060104804684E
:1001F0001048E4B244541068114A116804220139CD
:10020000884203D28021C9050A6002E01A6000E03A
:10021000116008221A6010BD98020010040000400E
:10022000180000408C02001094020010C00400105E
:1002300008000040B004001090020010D00400102C
:10024000AC0400101B4B02211A6810B50A431A6057
:10025000194B20211A68041C0A431A60174B1849CD
:100260001A680A401A601868012210431860154B7A
:1002700018680140196019680A431A60124B6C2211
:100280001A60124B1249186805F092F9114A106071
:10029000114A1060022C02D1104BA0221A60104BA0
:1002A000802212021A6080234022DB0501201A609E
:1002B00010BDC046048004408080044030400440AB
:1002C000F8FCFFFF3440044018000040A404001074
:1002D000400D030014000040100000400C000040DE
:1002E00000E100E0034B1B689A06FBD5024B186047
:1002F0007047C0461480004000800040FFFFFFFFB1
:100300007FB5051C00200C1C01F0A8FA002801D0C4
:1003100002F0C6FE00262660281C2E60211C01F07B
:10032000CBFA301C01F09AFAB04207D002F0B8FEC6
:100330002660281C2E60211C01F0BEFA0C4B1B7895
:10034000002B13D00B4B2A6818680B49824203D14B
:1003500020680D68A84209D01A60236801A80B60C4
:10036000064902F0F9FC01A802F09EFD7FBDC046DF
:10037000940300104401001048010010D8560000FA
:1003800038B5051C0C1C281C211C02F09BF8024BE4
:100390001B68002BF7D138BD7002001008B502F0C1
:1003A000C5F808BD08B500230B60036001F084FAAE
:1003B00008BD000010B502F03BFE0D4B002019688F
:1003C00002F060FA002002F04DFA002002F02AFA52
:1003D000084B01241C60084B201C198802F00EF900
:1003E000201C02F0FBF8201C02F0D8F810BDC0461B
:1003F000A004001088020010A804001037B50C24D7
:100400000120032102F05EF8684601A9FFF778FF9A
:10041000009D002D02D1013C002CF1D1FFF7CAFF55
:10042000281C3EBD08B5002002F00CFA012002F0A5
:10043000C5F802F003FE08BD38B5051C0C1CFFF71B
:10044000B9FF064AF823DB000121D150281C211CEA
:1004500004F0D6F9FFF7E6FF38BDC046E00400100F
:1004600010B5041CFFF7A6FF201C04F097F9041C2C
:10047000FFF7D8FF201C10BD08B50020FFF7F0FFE4
:1004800008BD000008B5021C0249034802F058FCF0
:1004900008BDC046EE560000E6560000F0B5314BF0
:1004A00085B01B68051C019304D0002B02D00020EE
:1004B00001F032FC01F044F82B4C2C482368022157
:1004C0000133032223602A4B01F028F92368013B02
:1004D000236001F03FF8FFF7CFFF2648FFF7D2FF78
:1004E000254F96239B003B6000243B689C4227DA03
:1004F00002F0E2FA002803D001F0A6FD002422E079
:10050000002D13D01D4EFA218900306805F050F8F7
:100510006423584301F0F0FF01F060FEFA213068D7
:10052000890005F045F801F0E7FF02E00A2001F03C
:10053000FDFF02A803A9FFF7E3FE029B002B02D0F8
:10054000002D02D107E00134CFE7019B002B02D040
:10055000012001F0E1FBFFF78FFF094802F0F0FBFB
:1005600005B0F0BD1000001004000010F3560000AC
:10057000346600000257000090030010A40400102D
:10058000085700001B4B73B5041C1B49186805F085
:100590000FF81A4900901A4A1A4B201C02F0DCFB93
:1005A00001F066FA002812D001F07EFAFA218900E3
:1005B000061C04F0FDFF051C201C02F01EFC124B63
:1005C00020186B431149F3182A1C02F0C5FB201CAC
:1005D00002F013FC0E4B20181B68002B02D003DA2C
:1005E0000C4A02E00C4A00E00C4A0D4902F0B4FB50
:1005F00073BDC046A404001040420F00195700000C
:10060000EE5600002657000018FCFFFF2A57000096
:10061000580100101657000013570000CF66000065
:100620003557000070B5051C0E1C141C00F088FF27
:10063000301C291C0022064B01F070F8201C0121FF
:100640000922044B01F06AF800F084FF70BDC04637
:10065000346600001C66000007B51449144A0120E6
:10066000FFF7E0FF642001F061FF72B6114B00213B
:100670001960114B01221A6019601A601968012271
:100680001142FBD00D4B68461A600D4B8022196851
:1006900052020A431A600B4B80211A680A431A60FF
:1006A0003923009301A9084B984707BD3D57000027
:1006B000CF6600007080044074800440788004405D
:1006C0008080044038820440F11FFF1F00B5084BB2
:1006D00089B01A78074B68461B78074902F03CFB43
:1006E00001206946054AFFF79DFF09B000BDC046DD
:1006F0004C010010080000106D5700007B570000EF
:10070000F0B52A4C2A4D237885B001932F78FFF756
:10071000DDFFFFF7B1FE002602A803A9FFF7F0FDF9
:10072000029800282BD0C0B201F016F840280CD057
:1007300004D830280ED0392817D01BE0462830D0F6
:1007400049280DD0412815D126E02B783E2B11D811
:10075000013303E02B78002B0CD0013B2B7009E018
:100760002378062B06D8013303E02378002B01D031
:10077000013B237000F0D0FEFFF7A8FF0026029B8C
:10078000002B02D0C82001F0D1FE04200321013645
:10079000FFF7F6FD1D2EBFDD019B2F70237000F0CB
:1007A000BBFEFFF769FE05B0F0BDC04608000010B3
:1007B0004C01001010B590B06846FFF7E3FE00F062
:1007C000BFFE084C012168460A1C231C00F0A6FF4E
:1007D000054801210922231C00F0A0FF00F0BAFE09
:1007E00010B010BD1C6600008F57000000B52D2210
:1007F0008DB0002800D02B2268460D4902F0ACFADB
:1008000004A802F0DFFC0120694604AAFFF70AFFF2
:1008100003200021FFF7B4FD0220FFF721FE00288E
:10082000EED00A200021FFF7ABFD0DB000BDC046A1
:10083000C8570000F8B5041C161C0D1C002702F058
:10084000C1FC211C1431E774681C02F0DFFA00F0CF
:1008500077FE201C04213A1C0A4B00F05FFF0A4C73
:10086000281C04210922231C00F058FFBE4205D099
:10087000064878210922231C00F050FF00F06AFE90
:10088000F8BDC046346600001C6600000867000022
:1008900010B58CB0FFF7F0FD124902A802F0B6FACD
:1008A00004A802A90022FFF7C5FF2E24FF3400226E
:1008B00004A802A9FFF7BEFF0020032101F002FEF9
:1008C0000023684601A901930093FFF719FD009BDF
:1008D000002B02D1013C002CE9D1FFF7CDFD0CB07B
:1008E00010BDC04660880000F0B5002493B00594A8
:1008F000FFF7C2FD0222962301940392271C5B009E
:10090000029300F01DFE019B9A4E002B6DD10AADA3
:10091000281C02F057FC019AEA742A746A73AA72BE
:10092000EA712A71002C01D1012F05D1281C042164
:100930000022331C00F0F2FE8F4D331C281C1E21B8
:10094000002200F0EBFE8B4E012C01D1012F06D1CD
:1009500068462D3025210022331C00F0DFFE281CC4
:1009600033210022331C00F0D9FE824D022C09D124
:10097000012F07D0684633304D2100222B1C00F098
:10098000CDFE09E00CA83A2100222B1C00F0C6FE87
:10099000032CEFD1012FEDD0784E2B1C301C5921A8
:1009A000002200F0BBFE734D042C01D1012F06D1B3
:1009B000684636305F2100222B1C00F0AFFE301C51
:1009C0006C2100222B1C00F0A9FE052C01D1012F67
:1009D00006D16846393072210022664B00F09EFE37
:1009E0000FA804210922664B03E066480421002277
:1009F000331C00F093FE00F0ADFD059B002B0AD0E8
:100A0000143B012B05D8052C03D0962001F08EFD58
:100A100001E0FFF731FD0320011CFFF7B1FC0020CE
:100A200000F01CFF0023051C06A905A806930593EA
:100A3000FFF766FC059B002B74D007AD08AE281CA1
:100A4000311C09AA02F0F2FB0190002871D1281C88
:100A500002F0D6FC071C05981238052868D804F067
:100A600045FD0567240C6703601C00E0601D06213E
:100A700004F0F4FD00270C1C5BE0601E042804D881
:100A800004F034FD060B0D103A002B88013316E0FC
:100A9000A8780C2104F082FD19E001375FE030787E
:100AA00001301BE07078013020E0601E042804D87B
:100AB00004F01CFD0810121A22002B88013B2B8029
:100AC000002445E0A8780C210A3004F0C7FD01316C
:100AD000A9703DE0013F42E030781730182104F062
:100AE000BDFD0422317040E070783B303C2104F0C1
:100AF000B5FD0323717030E00023B370381C07216B
:100B000004F0ACFD281C0A1C0991311C052C02D1F3
:100B100002F0E7FB02E0039B02F0A2FB0127962311
:100B2000BB4008E0002D07D101235F401F4003E0D8
:100B3000012796235B000293059B842B17D0182B6B
:100B400015D0029B029A013B002A00D0D8E60EE0A5
:100B5000281C02F055FC0523071C0393CEE7381C24
:100B6000291C02F07DFC022405220392C6E713B083
:100B7000F0BDC04634660000D1570000C6570000E3
:100B80001C660000D3570000F7B502F0B1FA182038
:100B90000021FFF751FC0024704DFFF743FC704E1D
:100BA000F8230022DB00F250201C02F0C2FA002CD5
:100BB00002D00020012101E00620032101F082FC87
:100BC000201C02F0B1FA01A9071C6846002F03D0CF
:100BD000FFF7E8FB012729E0FFF7E4FB009A002A72
:100BE00024D1002CE0D15F4B1B68002BDCD15C4B87
:100BF00098331B68002B0BD15B4BED18D4D500F05C
:100C000053FC574B002294331A600224534DCBE718
:100C1000564B00941A6811321A60009A102AEBDCC5
:100C200003F0A4FD009B01330093F6E7002C0BD0EA
:100C3000009B182B01D0002FAFD000F093FC4C4844
:100C4000FFF720FC0123F36600F040FF02F0BAF941
:100C5000009A182A69D1019F0024F8B200F07CFDA7
:100C6000F823DB0001250194F550192833D00FD863
:100C7000152835D007D811281ED0132852D1281C8A
:100C8000FFF70CFC51E0162832D017283BD049E082
:100C9000262830D006D8212815D0222842D104F0A9
:100CA00085F842E0442836D045283BD1E1200001B8
:100CB00002F030FB281C32E02E4B1B68002B34D096
:100CC000FFF7E6FD05E02B4B1B68002B2DD0FFF74F
:100CD0000BFE009429E0284B1868281A01F01CF834
:100CE0000120FFF767FDFFF7C7FBFFF787FB1CE05D
:100CF000FFF706FD19E0214B05221C70204B1A70EE
:100D000000F00AFC11E01F4B1A6801321A60072A32
:100D10000BD11C6009E01C4802F0FCFA201CFFF714
:100D200065FD02E000220197F250FFF743FB0098B7
:100D3000019903F065FDF823DB00F358002B01D087
:100D4000FFF79AFB064B94331B68002B03D100F08E
:100D5000ABFB012420E704F043FB1CE720BF0200AB
:100D6000E0040010700200100CFEFFFF9C02001057
:100D7000E157000058010010100000104C01001055
:100D8000080000101C010010F0F1FFFF73B54B4D7F
:100D90004B4B2A684B4C9A4202D12C6001F05AF816
:100DA0002B68A34202D1454B00221A60464C02F048
:100DB0006BF800F015FD4548002101F0DDF9002138
:100DC000434801F0D9F900F0E3FD00F083FF236808
:100DD0000726B3432360236801252B4300202360AB
:100DE000021C0B2101F052F9201C3A4C102101F099
:100DF000C3F923680022B34323602368281C2360BF
:100E0000042101F043F9201C002101F0B5F901F0A3
:100E100027F99620000201F0ABFD2F4D01235B4224
:100E200000202B60FFF7C6FC00232B60502401201C
:100E3000FFF708FA00F04EFF02F024F92B68002BB0
:100E400005D16420043C01F071FB142CEFD100208B
:100E5000FFF7B0FC2821214802F068FB142001F0C4
:100E600065FB1E48282102F061FB1D4801F068FF68
:100E7000192001F05BFB01F01FFE002803D00020C9
:100E8000FFF70CFB02E0013C002CF1DC15480821C7
:100E900001F072F902F0A8FB03F00CFB1E23009393
:100EA00010230193104811490022114B03F01CFB41
:100EB000104803F04DFBFFF767FEC0460800001026
:100EC000BE153E37E45BE173744004409840044033
:100ED0009C4004409440044058010010DE03000090
:100EE000EB570000104004405D5400000103000077
:100EF0009C02001088020010F7B500283BD0037850
:100F0000303B5A425341C0180378782B03D101304B
:100F10001026012501E00A2600250378002201920F
:100F20002D2B02D101230130019300230278002AE6
:100F30001BD0171C303FFCB2092C02D87343DB19BD
:100F400011E020273A43002D08D0171C613FFFB263
:100F5000052F03D81B01573A134304E0064801F05C
:100F6000EFFE002007E00130E0E7019A002A00D000
:100F70005B420B600120FEBDF55700000378202B7B
:100F800001D10130FAE77047031C303BDAB2092A7D
:100F900001D8181C0AE020231843031C613BDBB274
:100FA000052B01D8573801E001204042704770B549
:100FB0000E1CFFF7E3FF0025041C2078002807D053
:100FC000FFF7E2FF002803DB2D0105430134F4E7BE
:100FD0003560201C70BD000008B500F065FD011CE7
:100FE000014801F0ADFE08BD0358000000B589B00E
:100FF000684602F0E7F86946024801F0A1FE09B030
:1010000000BDC0463F580000F7B50F1C01A9161CD3
:10101000FFF772FF002814D0019C0B49201C04F03C
:101020001DFB0D1C081C642104F018FB281C3970E2
:10103000642104F0BDFA04493070201C04F0B8FAB1
:1010400001E001204042FEBD1027000037B50D1C15
:1010500048686A46694607310632FFF7D5FF01AC9A
:1010600069466A4620800132A8680231FFF7CCFF4A
:101070006B4618702288044B9A4203D9201C69469B
:1010800002F02FF937BDC0466B07000007B548686E
:1010900001A9FFF731FF019B3C20584302F03AF9C8
:1010A00007BD000007235843054A10189C30013B38
:1010B00004D3C25C002AFAD0002000E0012070476F
:1010C000E004001030B5194885B001F039FE002465
:1010D000651CA30719D1201CFFF7E4FF002810D0DE
:1010E000281CFFF7DFFF00280BD0A01CFFF7DAFF5A
:1010F000002806D0E01CFFF7D5FF002801D00434FB
:101100000EE00B48211C01F01BFE211C684602F07A
:101110007FFA684601F0D2FE064801F011FE2C1C51
:10112000FF2CD5DD01F0D8FE05B030BDEE56000035
:101130000F5800005F88000070B50E1CFFF71EFFFF
:101140000D25041C0134631E1878FFF71DFF0028CD
:1011500006DB7055013DF5D2201CFFF70FFF00E0C4
:10116000002070BD70B5444C86B023680868251C0B
:10117000002B06D1414801F0E3FD03F09BF9012368
:1011800009E0012B0DD13E49042201F048FE002860
:1011900003D12368013323606BE03A4801F0D0FDAE
:1011A0005FE00378412B17D1374C0230211CFFF749
:1011B000C3FF002855D00378422B52D1211C0230A6
:1011C0000E31FFF7B9FF00284BD00378432B48D1ED
:1011D000211C02301C3103E0532B06D12B49023075
:1011E000FFF7AAFF002844D13BE04D2B1FD1284C2C
:1011F0000230211CFFF7A0FF002832D003784E2BCD
:101200002FD1211C02300E31FFF796FF002828D085
:101210000378472B25D1023001A9FFF7C8FE019BB7
:10122000002B1EDB184A1B4853651B491DE001A912
:10123000FFF7BDFE04782023061C9C4311D1301C0F
:1012400002A9FFF779FF019B061CE118FF2902DCC8
:1012500002A802F0F3F9002E03D00134042CEED1E1
:1012600007E003F027F90B480C4901F069FD002362
:101270002B6006B070BDC0465C020010185800001C
:10128000EE5600002E580000E00400102605001065
:101290000A0500103A580000555700004458000055
:1012A00037B54C682378002B25D0201CFFF766FE4D
:1012B00001A9FFF77CFE019B041C002B1BD0D8B2B8
:1012C000FF2B09DD00F064FA019B051C1812C0B267
:1012D00000F05EFA019003E000F05AFA0025019058
:1012E0000198002802D0291CFFF7A6F823785A1E7F
:1012F0009341E418D6E737BD064A08B513780121B3
:101300004B40137001D0044900E00449044801F047
:1013100017FD08BD95030010E85700004B5800006A
:101320004F580000064A08B5137801214B4013704E
:1013300001D0044900E00449044801F001FD08BD62
:1013400094030010E85700004B5800005E5800005E
:1013500007B5486801A9FFF7CFFD019B002B01DC11
:1013600001230193019B1E2B01DD1E230193019993
:10137000962292004A43034B03481A6001F0E0FCB6
:1013800007BDC046900300106E58000008B50C4A17
:101390001378013BDBB21370002B0AD0012B02D172
:1013A0000849094A01E00949094A0A4801F0C8FC0C
:1013B00004E0094801F0C4FCFFF74EF908BDC0463F
:1013C0000000001092580000CF6600009658000000
:1013D000B96900009A580000BE58000038B5051CD5
:1013E000002D09D0642402200021013C00F074FE8D
:1013F000002CF8D1013DF3E738BD70B5061C012083
:101400000821021C00F092FE07240120082100227E
:1014100000F08CFE321C012522412A4000200221CE
:1014200000F084FE281C08212A1C00F07FFE013CED
:10143000EBD270BD10B50021041C0A1C022000F084
:1014400075FE201CFFF7D9FF10BDF0B5012385B054
:1014500002930023061C039372B6002402AB1B59AF
:10146000502040421843C0B2FFF7E4FF0020FFF7CE
:10147000E1FF1020FFF7DEFFE020FFF7DBFF212771
:1014800067430025F71902200021012200F04EFEDB
:10149000785D0135FFF7B1FF842DF4D10434082CB9
:1014A000DCD162B605B0F0BD08B5AC20FFF7C2FFD5
:1014B000AE20FFF7BFFFA520FFF7BCFF08BD38B582
:1014C0000122051C0C1C00F0E1FD281C211C01223E
:1014D00000F02CFE38BD08B5AF20FFF7ABFFA4200D
:1014E000FFF7A8FF08BD08B5AE20FFF7A3FF08BDB2
:1014F00010B5041CF820FFF79DFF201CFFF79AFF92
:1015000010BD10B5041C8120FFF794FF3F20204040
:10151000FFF790FF10BD000008B5074B20201B7897
:101520001843FFF787FF0A20FFF758FF034B18788F
:10153000FFF7E7FF08BDC046080000104C0100108F
:1015400008B5842202480021520001F033FC08BD96
:101550009603001008B50248FFF777FF08BDC046A4
:101560009603001008B501200821FFF7A8FF00200E
:101570000221FFF7A4FF02200021FFF7A0FF0220B5
:101580000621FFF79CFF0320011CFFF798FF0320B3
:10159000011C002200F0CAFD02200621002200F0FA
:1015A000C5FD06210122022000F0C0FDFFF7C8FFA3
:1015B000FFF7D0FFA220FFF73DFFA020FFF73AFF83
:1015C000C020FFF737FF0020FFF792FF0A20FFF748
:1015D00005FF4020FFF72EFF2C20FFF72BFF3220C6
:1015E000FFF7FCFE2E20FFF725FF3220FFF7F6FE67
:1015F0002F20FFF71FFF0A20FFF7F0FEFFF78CFFF9
:10160000FFF769FF08BD000083280ED80F290CD80A
:10161000CB08842253430722C0181140034B802279
:101620000A41111C1A5C11431954704796030010AB
:10163000F7B55B18DBB20193019B994215D2842563
:10164000CC086C4307270F40802504193D41EFB2B9
:10165000A618B44206DA054D65192B7801343B43D0
:101660002B70F6E70131C9B2E6E7F7BD960300102B
:10167000F0B51E1C87B00592F27804915B68824237
:1016800001D2307845E0244AB478934205D1032250
:10169000041B54430192E4180CE0001B0022824218
:1016A00004DA1978013202315B18F8E71A789C1CC9
:1016B0005B780193A218002503922F1C019B9F4287
:1016C00026DA08220023029200937378009A9A4245
:1016D0001CDA029A082A06D1039B9C4218D00022E9
:1016E000257802920134EB0708D5049A009BB818BC
:1016F000059AC0B29918C9B2FFF786FF009B029AFB
:10170000013301326D1000930292DEE70137D5E715
:10171000019807B0F0BDC046D9580000F7B5041CC9
:101720000D1C161C1F1C01F068FB20180190019B6A
:101730009C420DD0832D0BD82078291C3B1C321CD9
:10174000FFF796FF034B01341B68C0182D18EEE716
:10175000F7BDC0460400001010B50021012204238B
:101760000A4C0C5D844203D118010243D0B20BE055
:10177000013B002B04D10132092A00DD1A1C04238D
:1017800001312829ECD1002010BDC046446600007C
:101790000F23020918408000031F00D52833511E73
:1017A0000020032906D8242B04DC04218A1A0249CC
:1017B000CB18985C7047C0464466000038B5051CDD
:1017C0000024054B291CE05C044B0134C01800F0D8
:1017D000D3FC0A2CF5D138BD8066000000400440DF
:1017E000F8B50D4F3C68002C15D11020FFF7E6FF2F
:1017F0000A4B0022E65C1B195D78301C291C00F0A6
:1018000045FC0234301C291C012200F08FFC142CF2
:10181000EED101233B60F8BD500100106C66000062
:1018200070B500240B4B0122E65C1B195D78301C5F
:10183000291C00F02BFC0234301C291C002200F073
:1018400075FC142CEED10020FFF7B8FF024B0022EC
:101850001A6070BD6C6600005001001038B5051CA0
:10186000FFF7BEFF002D09D007210122022000F062
:101870000DFC104B80211A688A431A6000200B214E
:1018800000F02AFC0124002805D000200B2100F0E4
:1018900023FC44424441002D09D0072100220220AC
:1018A00000F0F4FB034B80211A680A431A60201CE5
:1018B00038BDC046FC3F0250F0B587B0002602900C
:1018C0000120039104960596FFF7C8FFB04202D0AD
:1018D0001823049301260021284C00912078617878
:1018E000012200F0D3FB20786178002200F01EFC7A
:1018F000234B9D1D012E24DC6A782F78111C381C87
:10190000019200F0E9FB002808D100991D4AB300BC
:101910008A5C103369465A5001360BE028786978A2
:1019200000F0DAFB0028F0D0381C019900F0D4FB5D
:101930000028EAD0009A144B0132023D00929D42E9
:10194000D8D127786578381C291C002200F09EFB2E
:10195000291C381C012200F0E9FB0C4902348C429E
:10196000BCD10020864206D0049A029B05991A60D9
:10197000039A0120116007B0F0BDC0466C660000FC
:101980003C660000446600003A6600008066000085
:1019900008B50120021C0B2100F078FB01200B216F
:1019A000002200F0C3FB03200221012200F06EFBA5
:1019B00003200221002200F0B9FB08BD234B37B5FC
:1019C0001A6810218A431A60214B802219689201FB
:1019D0000A431A60051C0B210120002200F056FB6F
:1019E00001200B21002200F0A1FB1A4B9F211A6855
:1019F000194C8A431A601A6818491A60184B1868FB
:101A000003F0D6FD8023000218432A1C2060022127
:101A1000032000F08BFB142000F088FD2368FF22D8
:101A20009343236023680F4A134323600E4B1B68C4
:101A30000193019B002BF9DA22680C4B13402360C1
:101A4000FFF7A6FF01980004800D3EBD38820440D8
:101A5000808004409840044000C0014000093D00DF
:101A6000A4040010800000012CC00140FFFFFFF81B
:101A700010B50C4C2068002813DA00202060FFF716
:101A80009DFF0A280ADC0120FFF798FF0138C023D8
:101A9000FF385B00984201D801232360FFF778FFED
:101AA000206810BD0C00001008B5FFF7E1FF00280A
:101AB00001D1002007E00120FFF780FF011EF8D0D0
:101AC000014803F075FD08BD50BB120008B5FFF7D3
:101AD000CFFF00280AD0FFF7E7FFFA22031C0021FE
:101AE000C00FD2009A424841014B186008BDC04661
:101AF0005401001008B5074B02221A60064BA222BF
:101B00001960064B1A70A32258709A7000F00AFEF2
:101B100008BDC046D0040010AC040010C004001082
:101B200008B5064B02311960054B00221A60054BBF
:101B3000A2221A70587000F0F5FD08BDD004001004
:101B4000AC040010C004001070B5051C0E1C03246A
:101B5000281C311CFFF7CEFF0223FF33984202D02E
:101B6000013C002CF4D170BD70B5051C0E1C032483
:101B7000281C311CFFF7D4FF0223FF33984202D008
:101B8000013C002CF4D170BD0B4B10B51C68002338
:101B90009C420ED0094CA31CA270140A5C70140C59
:101BA000120EDA709C70FFF7DFFF831EFF3B5A4274
:101BB0005341181C10BDC04658010010C00400104D
:101BC00070B50E4C25680024A54215D00C4C160AA1
:101BD000A270E670160C120E6271A371A21D26711E
:101BE0001C0A54701C0C1B0E9470D370FFF7BCFFC2
:101BF000841EFF3C63425C41201C70BD58010010F4
:101C0000C004001008B5064B1A6800239A4205D09C
:101C1000FFF79AFF831EFF3B5A425341181C08BD31
:101C20005801001008B5074B00201B68834207D0FD
:101C300002200721FFF788FF0238FF38434258414E
:101C400008BDC0465801001038B50F4B051C1B6875
:101C50000020834217D00924641B631E062B10D872
:101C6000072C05D00948A91E0918221C01F080F88C
:101C7000E8B2211CFFF778FF0238FF384342584191
:101C800001E00120404238BD58010010C20400109C
:101C9000012010B5011CFFF757FF0223FF339842C4
:101CA0000ED1094B01211960084B1C78230709D07C
:101CB000074B032222409A70081CFFF755FF01E0F2
:101CC00001246442201C10BD58010010B004001013
:101CD000C004001008B5FFF7DBFF02200121FFF769
:101CE00033FF0223FF3398420FD1084B1B787F2B21
:101CF00006D98422022007215204054BFFF760FF1A
:101D000009200421034AFFF73FFF08BDB00400107B
:101D1000020114008080808010B500280CD0254B73
:101D200080211A688A431A60234B1B68D907FBD5A8
:101D3000224B03221A6001E0204B1860204B012245
:101D400000211A6019601A60196801221142FBD043
:101D50001C4B80211A601C4A4902146821431160FF
:101D60001A1C002804D1134B8024196821431960E0
:101D7000164B196888421CD01860002801D01448FE
:101D800000E01448116803F0C5FB134BFA211860FA
:101D90008900041C03F00CFC1E2358430F4BC82180
:101DA00018604901201C03F003FC0D4B186001F082
:101DB00055F810BD388204400C8004407080044007
:101DC000748004407880044080800440100000103B
:101DD000006CDC02001BB700A4040010A00400107B
:101DE000A804001008B500F043F9134B00211A684D
:101DF000120B12031A60114B1A68120B12031A60AD
:101E00000F4B1A68120B12031A600E4B1A68120B52
:101E100012031A600C4B012219600C4B1A601960F6
:101E20001A601A68D107FCD5094B23221A600020DA
:101E3000FFF772FF08BDC0460080005000800150CF
:101E400000800250008003504080044044800440E1
:101E500008800440014A024B1A60FEE70400FA05BC
:101E60000CED00E038B50C490C4800F069FF0C4D52
:101E70000024281C00F064FF0A4A0B48A1581219DC
:101E8000D2682B1C143400F05BFFF02CF4D107480F
:101E900000F056FF38BDC046EE5600008A660000CE
:101EA000CD660000146800009C660000A766000074
:101EB000F0B5404B8BB01E68041C002E01D1351CC0
:101EC0000AE03D4B02901B6801209B6802A99847DD
:101ED0005EE033681E79019D2378002B31D0082DF8
:101EE00033D02378202B01D10134FAE7002B28D0FE
:101EF0006A1CAD0008356B460192EC50FF2E54D0A1
:101F00002278002A07D0631C202A01D01C1CF7E786
:101F1000002222701C1C019A012ADCD1264E274B7C
:101F20000D253360371C013D002D36D03B680298EB
:101F3000196800F085FF0028CBD03B6814333B6064
:101F4000F1E7002D24D0022D02D0B54206D911E0D0
:101F500003981B4900F074FF0028F6D1164C19486D
:101F60002368D96800F0ECFE23681748196900F06F
:101F7000E7FE0DE0104CE8B2236802A99B68984781
:101F800023689A68114B9A4202D0114B03221A70AF
:101F9000084A1368002B0BD103E0281C291CFFF70B
:101FA00061FF0C4800F0CCFE02E0019D0026CAE76C
:101FB0000BB0F0BD5C020010640200101468000059
:101FC00017570000C96600003F5800008D1300003D
:101FD00000000010D066000038B5041C164D0A2819
:101FE00008D002D8082811D01CE00D2802D07F2884
:101FF0000CD017E02A6800231370104800F0A0FEF0
:102000000F4C201CFFF754FF2C6013E00C4B2A6888
:102010009A420FD90B48211C00F092FE2B68013B1D
:102020002B6007E00748211C00F08AFE2B685A1C31
:102030002A601C7038BDC04660020010CD660000EA
:102040005C010010DC66000008B500F035FD0028DA
:1020500004D000F007FDFFF7BFFFF6E708BD000062
:10206000014A024B1A6070475C01001060020010C8
:10207000044B40211A680A431A60034B01221A706C
:102080007047C04680800440680200100F4B70B556
:102090001B78061C0C1C151C002B01D1FFF7E8FF58
:1020A000701E022803D80A4B8000C35800E0094B79
:1020B0001A68012D04D1A5402C1C14431C6003E0B8
:1020C0000121A1408A431A6070BDC0466802001019
:1020D000046900000080005038B50F4B051C1B78C8
:1020E0000C1C002B01D1FFF7C3FF0020032D12D8D9
:1020F000281C012203F0FAF902040608074B04E049
:10210000074B02E0074B00E0074B1B68A24013405F
:10211000181C421E904138BD68020010FC3F005060
:10212000FC3F0150FC3F0250FC3F03500F4B70B589
:102130001B78061C0C1C151C002B01D1FFF798FF07
:10214000701E022803D80A4B8000C35800E0094BD8
:102150001A68012D04D1A5402C1C14431C6003E017
:102160000121A1408A431A6070BDC0466802001078
:1021700010690000FC3F005038B5084B041C1B7868
:102180000D1C002B01D1FFF773FF23681822934326
:10219000236023681D43256038BDC04668020010D7
:1021A000054B3F221A60054B01221A60044B402167
:1021B0001A688A431A60704724800440D88004401B
:1021C0003882044008B5044B40211A688A431A60DB
:1021D000FFF7E6FF08BDC04638820440094B0A4AB3
:1021E00019680A40802149000A431A60074B0421FC
:1021F0001A688A431A60064B1A68064B1A6030BF89
:102200007047C04600800340FFF7FFFF10ED00E07D
:10221000388204403482044008B500F049FAFFF7E0
:10222000FFFA0A480021FFF7A7FF09480021FFF73E
:10223000A3FF08480021FFF79FFF07480021FFF791
:102240009BFF06480021FFF797FF08BD08400440A8
:1022500000400440AC400440144004401C40044092
:1022600008B50120FDF7EEFF08BD000008B5124BD0
:102270008022DA675200DA678022D200DA67802291
:102280005201DA6780221201DA6780229200DA674F
:102290000A4A002313600121094A49421160094A90
:1022A0001360094A1360094A01231360084A136046
:1022B000FFF7D6FF08BDC04604E100E004820440F9
:1022C0000882044004C000403CC0004000C0004000
:1022D0000040014008B5064B1A6801321A60054BF0
:1022E0001868FFF719FDFFF7C1FFC046C04608BDDB
:1022F0006C02001010000010F7B5071C0C1C72B621
:10230000FFF78AFF524B1A68524B1A60002F01D018
:10231000514B00E0514B524A04211360514B524D36
:102320001A680A431A6000232B60A1071ED04F4B86
:102330004F4A19680A401A6029684E4BA2070ED509
:10234000EC2252010A432A6080221A6052001A606D
:102350008022D2001A60802252011A6003E080229B
:1023600012010A432A60802212011A60002F53D002
:10237000414B00241C60414B414E1C60414B301CC2
:102380001C60414B211C1C60FFF7F6FE201C09213C
:10239000221CFFF77BFE201C0921221CFFF7C6FE32
:1023A0003A4B80211A683A480A431A603368072278
:1023B0009343336033680222134333600A21784326
:1023C00003F0A8F8334B03221860334B1C60334BE7
:1023D0001A60334B334A19680A401A601A68802120
:1023E0000A431A60234A8B001360204A116819437C
:1023F00011602A68022113432B602B4B01221A60C3
:102400002A4B19602A4B1C491A601C601A60186814
:1024100001221042FBD00A60264B012252421A6070
:10242000254B00221B680193244B1A6062B630BF13
:10243000C046214B019A1B689A4208D11F4B0122CA
:102440001A601F4B1868FFF767FCFFF70FFFF7BD17
:102450003882044034820440BF180000FF18000096
:102460003082044010ED00E0048204400082044009
:102470007FE2FFFF00E100E004C0004004000140F3
:1024800064400440044001400480014080800440D6
:10249000841E000018C0004008C0004014C0004066
:1024A0003CC000400FF0FFFF788004407080044083
:1024B00074800440088204406C0200107002001016
:1024C0001000001008B5FFF717FF08BD074B1A688A
:1024D000013203D1064A1168013111601A680132D4
:1024E0001A60044B1A6801321A60704780020010AB
:1024F0007C02001074020010074B98420AD8074A69
:1025000000231360064A01381060064A1360064B28
:1025100007221A607047C046FFFFFF0080020010CC
:1025200014E000E018E000E010E000E00B4A10B515
:102530001368002800D10120C1438B4208D91168DB
:10254000994209D3591C146809188C42FAD3F6E74A
:102550001168C91A8142FBD310BDC0468002001029
:10256000014B18687047C04680020010034B0122DF
:102570001A60034B1A6801321A60704700C00040AD
:1025800084020010034B01221A60034B1A680132C7
:102590001A6070470000014088020010002803D133
:1025A000044B01221A6003E0012801D1024B18609C
:1025B0007047C04604C0004004000140002802D11A
:1025C000044B186004E0012802D1034B00221A607A
:1025D0007047C04604C0004004000140002801D1FB
:1025E000044B02E0012804D1034B1A6802210A437C
:1025F0001A60704704C000400400014010B5002973
:1026000000D1134900280DD1124B80241A682243AF
:102610001A60114B03221860104B1960104B1A609E
:10262000620211E0012811D10A4B80221868520081
:1026300002431A600B4B00221A600B4B03221960F5
:102640000A4B1A6080229202094B1A6010BDC046E4
:10265000FFFF0000808004408402001018C000408A
:1026600014C000408802001018000140140001400E
:1026700000E100E080231022DB051A60094B0822EC
:102680001A6000238022D2051268D10604D5064ABA
:10269000934201D00133F5E7044898429B415842E8
:1026A0007047C04618000040FF0F0000FE0F0000FA
:1026B00008B58022154B1202DA67154B6C221A609E
:1026C000144B154A196800201140196019681960E7
:1026D000124B19680A401A601A6804211A60012214
:1026E000FFF7D4FC002004210122FFF71FFD00208A
:1026F00005210122FFF7CAFC012200200521FFF776
:1027000015FD074B00221A6008BDC04604E100E039
:102710001800004030400440F8FCFFFF3440044003
:1027200004800440F8B5174A174C00232360136057
:10273000164A202113608022D20511602168144AB4
:10274000012903D0934203D00133F7E7934203D129
:10275000FFF790FF002014E00E4F00253E68013E79
:102760002368FF2B0CD83B689E4204D03E68FFF7DD
:10277000F7FE051C0A35FFF7F3FE8542F0D1E7E7C7
:102780002068F8BD8C020010900200109402001026
:10279000FF0F000098020010034B01221A60034B48
:1027A0001A6801321A607047004001409C02001014
:1027B000174B70B501241C60164B1A6812191A6069
:1027C000154B1A68002A22D01A68144D013A1A6073
:1027D0001E68002E0DD02A68201C211CFFF7A6FCC5
:1027E0002B68201CE31A2B602A680221FFF79EFC4D
:1027F0000DE01B68201C2B602A68211CFFF796FC4B
:102800002A68201C0221FFF791FC054B1E6070BD59
:1028100000800140A4020010A0020010A8020010D5
:1028200004800140002803D1044B01221A6003E018
:10283000012801D1024B18607047C0460440014096
:1028400004800140002802D1044B186004E00128F4
:1028500002D1034B00221A607047C0460440014079
:1028600004800140002801D1044B02E0012804D17A
:10287000034B1A6802210A431A6070470440014062
:102880000480014010B500280FD1124B80221C6833
:10289000920022431A60104B032218600F4B1960FC
:1028A0000F4B1A608022D20211E0012811D1094B8E
:1028B00080221868D20002431A600A4B00221A6074
:1028C000094B03221960094B1A6080221203084B3E
:1028D0001A6010BD808004409C0200101840014026
:1028E00014400140A40200101880014014800140EF
:1028F00000E100E008B5184B1A680E231340062BC0
:102900000DD1164B9E221B68134205D0144ADBB230
:102910005360144B1B681EE0D9071CD501E0042B43
:1029200005D1104B1868C0B200F0B1F813E00C2BC1
:1029300006D10B4B8022596852000A435A600AE0C4
:10294000022B08D1054B1A68054B910601D50022D0
:1029500000E001229A6008BD088000401480004019
:10296000AC0200100080004000487047AC0200102C
:10297000F7B52D4B2D4C8022002192030191061CAE
:10298000DA67201C902200F015FA019B0725A3604E
:10299000274B284F1A68AA431A601968012211436D
:1029A0001960254B1968A94319601968114319600A
:1029B000224B80211868490101431960204B1A609D
:1029C00083223A601F4A126819681F4B18685043E7
:1029D00002F0A0FD311C000902F09CFD1B4B1022EF
:1029E0001B491A60030A0B601A4BC0B2032218601D
:1029F0003A60194A1560194A1D1C10680190106848
:102A000060230340602BFAD110680123184202D0E2
:102A10002B680193F8E723708022114B92031A6010
:102A200005230B60F7BDC04604E100E0AC020010D6
:102A3000A44004400C800040A84004408080044032
:102A40009880044078800440A4040010288000404E
:102A50000480004000800040088000401480004056
:102A600000E100E008B5FFF77FFFC268031C120217
:102A7000120E8218D07BDA681202120E0132D2B224
:102A80009A7352B2002A01DA00229A7308BD10B577
:102A9000041CFFF769FFC2681204120E8218D47377
:102AA000C2681204120E0132D2B2427352B2002A2C
:102AB00001DA0022427310BD08B5FFF755FFC26866
:102AC000C36812021B041B0E120ED01A431E98413B
:102AD000C0B208BD70B500241D5D0619002D02D0DE
:102AE00005550134F8E7121B301C131C002B03DDC5
:102AF0000170013B0130F9E7D043C0170240A01834
:102B000070BDF7B5051C01910093561E092B01D825
:102B1000041C0CE000980A2102F0FCFC0199031C43
:102B2000321C281CFFF7EDFF071C2C1807E0671B61
:102B3000002E04DD019B013E23700134F7E700986D
:102B40000A2102F02BFD3031781C2170FEBDF8B552
:102B50000C1CD9175F18051C4F40561E092F12D99F
:102B6000381C0A21002B03DA02F0D4FC434202E0B5
:102B700002F0D0FC031C281C211C321CFFF7E7FFCD
:102B8000041C2D1814E0002B00DA961E2A1CA9192B
:102B9000891A002902DD14700132F8E7F443E417C2
:102BA00034402D19002B03DA2D232B70013401350D
:102BB000381C0A2102F0F2FC30312970601CF8BD8B
:102BC000F7B5089F1E1C051C013A3B0901D1041CE6
:102BD00005E00093331CFFF7F3FF2C1806E0601BA1
:102BE000002A03DD2170013A0134F8E70F231F406A
:102BF000092F01D8303704E0002E01D0373700E02C
:102C0000573727700130FEBDF0B585B0041C029126
:102C100001D00021017000251178002906D1029F02
:102C20000023BD426CD22370281C6FE0029FBD427E
:102C3000F5D2252902D00132217004E051782529EE
:102C400004D12170023201350134E5E7302902D088
:102C5000561C202100E0961C32782D3A5042424109
:102C6000B6180022307830277F423F18FFB2092F74
:102C700007D80A277A438218D2B2303AD2B2013644
:102C8000F0E7AF18BC46029FBC4501D97A1BD2B20F
:102C9000692818D00BD863282AD0642813D0582864
:102CA00032D11F1D1B68201C009301231DE07528D5
:102CB0000FD0782814D0732826D11F1D201C1B6824
:102CC000FFF708FF0AE01F1D201C1B68FFF73FFFEE
:102CD00004E01F1D201C1B68FFF713FF3B1C0BE0CB
:102CE0001F1D1B68201C00930023FFF769FFF5E7F9
:102CF0001868043320700120721C24182D188BE7EB
:102D0000013C2370681E01E00120404205B0F0BD87
:102D100010B50C1C131C6421221CFFF775FF10BD9D
:102D200000B5031C9BB00A1C01A8191CFFF7F0FF9B
:102D3000632800DDFEE701A800F0B6F81BB000BD77
:102D40000FB407B504A908C9181C0191FFF7E8FFE3
:102D500003B008BC04B018470EB403B503AA08CAF0
:102D6000191C0192FFF7D4FF02B008BC03B018474A
:102D700030B50C1C044303232340041C002B01D05A
:102D8000002310E0032AFBD9CC58C4500433D41AD2
:102D9000032CF9D8131F9B0801339B00C418C918D2
:102DA00003231A40ECE7934203D0CD5CE554013392
:102DB000F9E730BD30B5031C840701D1032A01D8DF
:102DC0009A1814E00B060C041D1C25430D430C023D
:102DD0002543031C20C38418E41A032CFAD8131FBC
:102DE0009B0801339B000324C3182240E8E7934269
:102DF00002D019700133FAE730BD021C031C981A87
:102E00000133591E09780029F9D17047031C0A784B
:102E10001A70002A02D001310133F8E7704730B54B
:102E20000023934208D0C45CCD5C651B06D10133FE
:102E3000002CF6D1201C02E0002000E0281C30BD50
:102E400010B50022835C8C5CA34204D10132002BBC
:102E5000F8D1181C00E0181B10BD000008B5094B84
:102E6000FA211868890002F0A3FBFFF745FB9620C2
:102E70000002FFF77DFD0120FDF7E4F9FEF72AFFD0
:102E800008BDC046A404001008B5FEF7ABFFFFF76D
:102E9000EFF8FFF797F9FEF765FBFEF751FBFFF739
:102EA000DDFFFFF7DDF808BD10B5041C2078002811
:102EB00003D00134FDF716FAF8E710BD38B5051C4C
:102EC0000E24013C04D3295D0248FFF739FFF8E7DF
:102ED00038BDC0461C69000038B51948FFF730FFFF
:102EE000184C201CFFF7EAFF174D4221281CFFF762
:102EF00027FF201C0E30FFF7E1FF4321281CFFF7BE
:102F00001FFF201C1C30FFF7D9FF1048FFF718FFE8
:102F1000201C4630FFF7D2FF0D48FFF711FF201CA1
:102F20002A30FFF7CBFF281C4E21FFF709FF201C9A
:102F30003830FFF7C3FF616D0648FFF701FF38BD6A
:102F40001F690000E0040010256900002C690000E2
:102F5000326900003869000003110A2253430F222E
:102F600010401818704738B50A21041C02F020FBE5
:102F70000A210501201C02F071FB281C084338BD02
:102F800008B5C12252000E200221FEF7FDFD024BC2
:102F900001225A7108BDC046D404001010B5084C77
:102FA0006379002B01D1FFF7EBFF23790C221A4341
:102FB000A37901205B001A43011CFEF7E5FD10BD5B
:102FC000D404001010B5074C2379002B08D1637985
:102FD000002B01D1FFF7D4FF01232371FFF7DEFFA0
:102FE00010BDC046D404001008B5054B1A79002A5C
:102FF00005D000221A711A72DA70FFF7CFFF08BDF0
:10300000D404001010B501210220FEF7FBFD064B91
:10301000041C18787F231840FFF79EFF034B58705D
:10302000DC71201C10BDC046B0040010D404001098
:10303000014B01229A707047D4040010024B002209
:103040009A701A727047C046D404001008B5FFF792
:10305000D9FF094B094A9978002908D0197A012922
:1030600001D8013103E010680549086000E01972D9
:103070000021D970116008BDD40400107402001042
:103080007802001008B5FEF703FE0C23184003D0A9
:10309000024B1A781043187008BDC046D4040010C3
:1030A00010B5FFF7EFFF054B1A781C1C530701D52D
:1030B000FFF7CCFF0023237010BDC046D4040010DE
:1030C00008B50020FEF7CAFB002801D0FFF7E8FF93
:1030D00008BD000010B5054C0023E371FFF7F0FFB9
:1030E000E379002B01D1FFF78DFF10BDD404001050
:1030F00008B50948092102F0BDFA084BFA22D200AE
:103100001A80FFF7E7FF064B00221A60FA22054BF0
:1031100092001A6008BDC046D4040010DE040010FE
:10312000740200107802001008B5FFF7C9FF0020F4
:1031300008BD08B5FFF758FF08BD000070B51D4C6D
:10314000061C637822781B021343A278A07912042C
:103150001343E2780D1C12061343174A13401A0A50
:10316000237062701A0C1B0EE3706379A2702279CF
:103170001B021343114A134023711B0A6371FFF7AB
:10318000EBFE0F4B1B88C01830806079FFF7E4FE20
:10319000B070E078FFF7E0FEF070A078FFF7DCFE9B
:1031A00028706078FFF7D8FE68702078FFF7D4FEAB
:1031B000A87070BDB00400107F7F3F3F071F000064
:1031C000DE040010F0B58DB0051CFEF72BFD0028C5
:1031D00004D1281C1249FFF7BFFD1EE00AAE0BAC5C
:1031E000211C301CFFF7AAFF3388F7780793B378C8
:1031F000267808936378A47809930A4B187900F02D
:10320000D7F8099B04900293009701960394281C19
:103210000549079A089BFFF79FFD0DB0F0BDC0461A
:1032200044690000B00400104969000070B5061C34
:103230000D1C141CFEF7F6FC00280AD0301C291CBB
:10324000FFF77CFF002C07D0044B00201B79236084
:1032500003E00120404200E0201C70BDB0040010DB
:10326000F7B504880E1C051C6421201C00920193F4
:1032700002F094F9114B8FB2B078E41B1C80FFF779
:1032800072FE0F4CA0707078FFF76DFEE070307822
:10329000FFF769FE2071E878FFF765FE009B60711B
:1032A000A371A878FFF75FFEE071381CFFF75BFEA3
:1032B00020720198FEF7C8FCFEBDC046DE04001077
:1032C000C004001008B50223FFF7CAFF08BD08B507
:1032D000021C501E8241520100200121FEF754FCC5
:1032E00008BD38B5041C01200D1CFFF7F0FF201CA1
:1032F00000F086F8072102F0B1F9201C0A1C291CF5
:10330000FFF7E0FF96204000FFF710F90020FFF7DD
:10331000DEFF38BD73B5041CFFF774FE002801D131
:1033200000203BE01E4B5D781E1C7378AB4207D13A
:103330000A20FFF7FBF8FFF765FE0028F5D1EFE75D
:10334000FEF770FC0028EBD001A96846FFF7F6FEF7
:10335000684600F055F8051C01A800F031F8114B43
:1033600004199C420DD9E31701221343ED18281CC0
:10337000694600F075F8002C01DA0B4B00E00B4BAE
:10338000E418201C01A900F024F8281C072102F0F1
:1033900065F968460A1C01A9FFF794FF76BDC0468F
:1033A000D40400107F5101008051010080AEFEFF67
:1033B00007231840014B8000C0587047BC690000CB
:1033C00002783C235A434178521853438278981824
:1033D000704738B50C1C3C21051C02F03FF9281C35
:1033E000A1703C2102F0E4F83C2102F037F9617051
:1033F000E121281C090102F0DBF8207038BD000033
:1034000070B58378022100229942524104889621A6
:103410004901051C64180C20A41A42439B18033B65
:10342000992058430521023002F0C2F86E26FF367B
:1034300066436421A31086194942201CF61802F045
:10344000B7F8C82136184900201C02F0B1F8034B28
:103450003018C018EB78C01870BDC046D382FFFF8B
:10346000F8B5204B0C1CC5181F4B8000C0181F4915
:1034700002F09EF803235843C617B60F3618B6104D
:10348000AE19B600953E301C194902F0E7F8CD1789
:10349000AD0F6D180527AD107D430235281C99210D
:1034A00002F0DCF8081C391C02F082F80130E070F0
:1034B0009921281C02F07CF80C21023002F0CEF891
:1034C0004D1CEDB2A570301C094902F071F8094B92
:1034D0000C21C6180E20401B02F06AF83618268010
:1034E000F8BDC04679050000652F0400B13A02001E
:1034F000B505000094EDFFFF012008B5011C021C7A
:10350000FEF714FE0120021C0221FEF70FFE01202F
:10351000011C0022FEF7BAFD012002210022FEF765
:10352000B5FD0120FFF78EF908BD0000194B70B5FD
:103530000D1C196807229143196019680124214361
:103540001960154B061C1968201C914319601A68F4
:10355000211C22431A60221CFEF798FD221C201C0D
:103560000221FEF793FD0D4B311C186802F020F884
:10357000011C201CFFF786F9201CFFF773F9084E89
:10358000201C3560FFF74EF93368002BFCD1FFF7A4
:10359000B3FF70BD7C40044080400440A404001090
:1035A000A0020010F8238A01DB0013404A05920EA6
:1035B0001343F8221202114019430A23594330B52C
:1035C000CA1083181C1CEB345D782478EA336C40F5
:1035D0001B7824021C43835C201C5840072319409D
:1035E00008418005800D30BD7047000008B5054BCF
:1035F000011E994201DD044BC1180448EA38FFF767
:10360000D1FF08BDFF17000000F8FFFFF8690000B8
:103610000723594310B5084B59189C310023CC5C43
:103620000F2222400270CA5C01331209427002303C
:10363000072BF4D110BDC046E00400100723594306
:1036400010B5074B59189C310023427804781201B9
:103650002243CA5401330230072BF6D110BDC046B5
:10366000E004001070B5AC4C86B0E36E6E465A1E96
:10367000934117363370A94BE258D006400F0138FA
:10368000062807D801F032FF040C2012181A1D007A
:10369000022509E0636E16339B001B591D1C15E0C3
:1036A000636E16339B00E55800230FE0A36DE56DB4
:1036B000AB420BDD0D2509E0022503E00C250323B9
:1036C00004E00D252B1C01E00D25EDE750111F280E
:1036D00000D91BE101F014FF2000220029002C007A
:1036E0002F0033003B00440048004C0054006100B0
:1036F0006E00760083008F009B00A800B800C50014
:10370000D500D300E100E400E700EF00FE00020175
:103710000B010D010F011501E01801E0E0180E305A
:10372000EB1A591C01F0A6FFF0E0E0181C30F7E797
:10373000211C0E3105E0E0180E30E1180BE0211CD1
:103740001C31201C1A1C2B1C01F067F9DEE0E0186C
:10375000E1181C300E31EB1A5A1CFFF709FBD5E0BB
:103760006F48011C0E31EDE7E018011C1C31F2E737
:10377000226E1021002A00D00A21221C0E3206E0FF
:10378000226E1021002A00D00A21221C1C32029134
:1037900000950196201C211C53E0216E01223270FD
:1037A0001022002900D00A22009501960292201CC6
:1037B000211C45E0226E1021002A00D00A21221C83
:1037C0000E3213E0216E012232701022002900D047
:1037D0000A22009501960292201C211C4DE0226EC7
:1037E0001021002A00D00A21221C1C3200950196CB
:1037F0000291201C6AE0226E1021002A00D00A21CA
:10380000484A029100950196101C111C19E0216E86
:103810001020002900D00A20424A0290111C1C39B5
:1038200000950196101C0CE0216E012232701022CE
:10383000002900D00A223B49009501960292081CFB
:10384000002201F0F4F861E0226E1020002A00D07E
:103850000A20344A0290111C1C3900950196101C54
:1038600035E0216E012232701022002900D00A2298
:103870002C49009501960292081C002227E00122A3
:103880003270226E1021002A00D00A21254A0291AE
:1038900000950196101C002119E0009620481BE0BD
:1038A0000096204818E0226E1021002A00D00A213C
:1038B000221C1C3206E0226E1021002A00D00A21B0
:1038C000221C0E320095019602910020211C01F06D
:1038D000D6F81BE00096201C002103E0211C1C31BF
:1038E0000096201C1A1C2B1C01F02CF90EE0201C49
:1038F00002E00B4800E00B48191C2A1C01F039F9C2
:1039000004E0201C191C2A1C01F03DF93378012029
:10391000E36606B070BDC046E0040010C4070000B6
:10392000EE040010FC040010064B10B51A1DD46FF5
:10393000191C0831CC67D96FD1679A6F9867DA671D
:1039400010BDC046E0040010064BD96F1A1D986FD9
:103950009967D16F08335967D96FD1670022DA6749
:103960007047C046E0040010F8B5134C261C8C3696
:1039700030680130FFF73AFEF923DB00E0500F4BCF
:103980000122E758A36E051C02409A4211D1830719
:1039900003D430680230FFF7C7FFFF2292001540C2
:1039A000231CAD01BF108C332F431F60044B012239
:1039B000E2500220F8BDC046E0040010C407000039
:1039C000AC0700000F4A104B30B5D158131C8C3394
:1039D0001C68CB059B0E01208D0501D5403B02E004
:1039E000002B00D1031C89100840916E884206D13B
:1039F000111C8C31E3180B60044B0121D1500120C4
:103A000030BDC046E0040010C4070000AC07000051
:103A100008B5084B5A1CD07F9A1CD27F00011202B5
:103A2000104303331A7FDB7F10431B031843FFF758
:103A30007BFF08BDE004001008B5FFF785FF0323F6
:103A4000044A0F219A180140013311770011072B06
:103A5000F6D108BDE004001008B5FFF775FF044B70
:103A600001211A1C8C321060024A995008BDC046D0
:103A7000E0040010AC07000010B5064CA36E002B4C
:103A800007D0FFF761FF231C8C331860024B012223
:103A9000E25010BDE0040010AC07000010B5064C69
:103AA000A36E002B07D1FFF74FFF231C8C33186048
:103AB000024B0122E25010BDE0040010AC070000F0
:103AC00008B5054A054B0121D150054B1B68002B59
:103AD00000D0984708BDC046E0040010BC070000B5
:103AE0003C03001038B5154A154B00209850F822B9
:103AF000D2009A5882421AD0F622D20099588142B6
:103B00001ADD012909D1F721C9005C58844204D08B
:103B10000C4D58500A215C5199509A58032A01DDE6
:103B20000121D966F621013AC9005A5004E0064B3A
:103B30001B68002B00D0984738BDC046BC0700006A
:103B4000E0040010B40700003C030010094BF82209
:103B5000D2009A58002A04D0F622D2009A58002A9D
:103B600007DD054A0F219A58013311409977121148
:103B7000DA777047E0040010B4070000044B597F67
:103B80009A7F090112020A43197F0A435A67704754
:103B9000E00400100B1C093B30B5012B0FD80023AB
:103BA000074A9C18257FC45CA54205D0054B0839FF
:103BB000D0580143D15002E001330E2BF0D130BD7B
:103BC000E0040010A407000008B508290DD0192949
:103BD00013D1427808231A4202D00022027002E078
:103BE0000F2303700723437005E000230022C25413
:103BF00001330E2BFAD1FFF721FD08BD30B5114D71
:103C000085B06C6F002802D00F239C4304436C677F
:103C1000FF2C05DD281C1C300E2101F02BFD0FE0D0
:103C20006846211CFFF7F4FC6846211CFFF7CCFF17
:103C300000236846C15CEA18013311770E2BF8D1D6
:103C400005B030BDE0040010134B30B5596F0F22A2
:103C50009143041C0C4385B05C671D1C082C19D0D3
:103C6000FF2C17DC6846211CFFF7D2FC6846211C9C
:103C7000FFF790FF0023EA18127F6946CA54013308
:103C80000E2BF8D16846211CFFF79EFF6846211CC9
:103C9000FFF7D4FC05B030BDE00400101FB50F4C99
:103CA000616F082918D0FF2916DC6846FFF7B0FCC1
:103CB0006846616FFFF76EFF0023E218127F6946C6
:103CC000CA5401330E2BF8D16846616FFFF77CFFB1
:103CD000616F6846FFF7B2FC1FBDC046E0040010EC
:103CE00010B50D4C631CD87FA31CDB7F00011B02A9
:103CF0001843E37F1843E31CDB7F1B031843FFF7E4
:103D000075FC0F23021C1A40227702111340001287
:103D10006377A07710BDC046E0040010044B5A6ED4
:103D200016329200D258121A51424A41DA6670474E
:103D3000E0040010044B5A6E16329200D15801393B
:103D400000D50D21D1507047E0040010054B5A6E8C
:103D500016329200D15801310E2900D10021D150E4
:103D60007047C046E0040010144B10B55A6E191C81
:103D700016329200D2580C2A05DC9A18507F117F17
:103D80000001021C17E00E48F5241858A400A042B8
:103D900005D00C4C2040B724A400A04207D18A18BB
:103DA000137F486D1B01021113434B6505E09A1800
:103DB000127F197F12010A435A6510BDE0040010FA
:103DC000CC070000FFFEFFFF264B10B55A6E1632DF
:103DD0009200D2580C2A05D123495858F521890060
:103DE000884204D0FA21C900595800290DD0596DD4
:103DF0000F240C409A180811107754770901FF22FC
:103E0000114008431C7758652BE00C2A07DC596DDC
:103E10009B180F220A4009111A77597721E0124A9C
:103E2000F5219A5889008A4205D010490A40B721E5
:103E300089008A420DD15A6D0F20191C104029317A
:103E400008701001FF2108401111021C0A435A6535
:103E500007E05A6D191C1011293108700F210A4012
:103E60001A7710BDE0040010CC070000FFFEFFFF32
:103E7000244B0F215A6E586D16329200D2580140D1
:103E800070B500110C2A05D11F4C1D59F524A40052
:103E9000A54204D0FA24E4001C59002C09D09C1837
:103EA000657F267F2D0135435D651D7F2077657712
:103EB00026E00C2A08DC9C18657F267F2D013543FF
:103EC0005D65607721771CE00F4AF5249A58A400BD
:103ED000A24205D00D4C2240B724A400A24207D133
:103EE0001A1C29321478117024012043586508E007
:103EF0001A1C293214781D7F24012C435C65107034
:103F0000197770BDE0040010CC070000FFFEFFFF32
:103F100008B503480E22011C1C39FEF729FF08BD15
:103F20001805001008B503480E22011C1C31FEF7CD
:103F30001FFF08BDFC04001008B504480022011C46
:103F40001C310D2300F069FD08BDC046FC040010C3
:103F500008B503480E22011C0E39FEF709FF08BD03
:103F60000A05001008B503480E22011C0E31FEF7A9
:103F7000FFFE08BDFC04001008B504480022011C27
:103F80000E310D2300F049FD08BDC046FC040010B1
:103F90000023044A00219A18463201331170082B7D
:103FA000F7D17047E0040010C31C421E002093426A
:103FB00007D004494000591846310978013B0843AD
:103FC000F5E77047E004001010B50B1D994208D0CA
:103FD000044A01248A18044046321470401001310A
:103FE000F4E710BDE004001038B50020FFF7DCFF57
:103FF000084C051C0021207FFFF7E6FF04202577F1
:10400000FFF7D2FF0421051C607FFFF7DDFF657716
:1040100038BDC046E004001010B50020FFF7C4FF13
:10402000034C20770420FFF7BFFF607710BDC04628
:10403000E004001010B5054C0021207FFFF7C4FFFD
:10404000607F0421FFF7C0FF10BDC046E0040010F0
:1040500010B50A4C231C8C3318680130FFF7C6FAE0
:10406000F923DB00E050021C0F231A4022770211D3
:10407000134000126377A07710BDC046E004001023
:1040800010B5084C0E21201C01F0F4FA201C0E3053
:104090000E2101F0EFFA201C1C300E2101F0EAFA8B
:1040A00010BDC046E0040010054B1A1C0E32197FEB
:1040B000187801330143D9769342F8D17047C0464E
:1040C000E0040010054B1A1C0E32187F19780133DA
:1040D0000140D9769342F8D17047C046E004001001
:1040E00030B5002185B00E4B421C1818007F6C467D
:1040F00008550D25D40F181C002395425C416442DD
:10410000013122400E2901D0101CECE76C46E15C25
:10411000C218013311770E2BF8D105B030BDC0465F
:10412000E0040010074B10B55A6E16329200D458B6
:10413000611E1C19D1502077002901DA0D21D150C0
:1041400010BDC046E0040010034A0023111C943146
:1041500098320B6013607047E0040010034B01229B
:10416000943319684A401A607047C046E004001052
:10417000074B0022191C8C310A601A67054A01217D
:1041800099501A1C9432126851424A41DA667047BB
:10419000E0040010AC0700009A4B9B4910B5CC58C6
:1041A0000F20A310994A1840A411013812570E2865
:1041B00044D801F09BF9080E151C20432643432DDB
:1041C000434343313500002A38DB8A18403200234C
:1041D00004E0002A32DB8A184032012393712BE07D
:1041E000002A2BDB8A1840329379CB6624E0201C0E
:1041F000FFF798FF20E0002A20DB101CFFF78EFD60
:104200001AE0002A1ADB4B6E16339B00CA5013E0EB
:10421000201CFFF719FD0FE0201CFFF7EFFC0BE05F
:10422000002A0BDB101CFFF75BFF05E00C2B20DDE9
:10423000162B25D1FFF798FD0120E9E0982B02D13C
:1042400000230B66F8E7982B69DC382B02D101209C
:104250004866DDE0382B2EDC1C2B02D1FFF758FE20
:10426000EAE71C2B11DC0C2BE0D19831012008600F
:10427000CEE00120002B00D1CAE001204042C7E07F
:10428000182BFAD1FFF774FFD6E7282B02D10023B1
:104290004B66D1E7282B04DC262BEED1FFF794FDEB
:1042A000CAE72C2B02D1FFF73DFEC5E7362BE4D140
:1042B000FFF7DEFDC0E7662B02D1FFF753FEBBE739
:1042C000662B16DC4C2B03D1FFF7C2FE02209FE0C9
:1042D0004C2B04DC3C2BD0D1FFF72EFEACE7562B49
:1042E00002D1FFF735FEA7E75C2BC6D1FFF790FBA5
:1042F000A2E76C2B02D1FFF79FFB9DE76C2B04DC40
:10430000682BBAD1FFF7BCFE96E7762B02D1FFF7F8
:1043100033FE91E7882BB0D1FFF718FC8CE7E62B32
:1043200002D1FFF779FE87E7E62B33DCC82B02D1F9
:10433000FFF714FF80E7C82B15DCA82B02D1012062
:10434000086665E0A82B04DC9C2B96D1FFF716FCD1
:1043500072E7B82B02D1FFF7F7FE6DE7BC2B8CD1CB
:10436000FFF79CFC68E7D62B02D1FFF763FE63E7FB
:10437000D62B04DCCC2B80D1FFF7B2FC5CE7D82B2A
:1043800002D1FFF779FB57E7DC2B00D075E7FFF789
:104390008BFE51E7F32B02D1FFF7A4FB4CE7F32B85
:1043A00017DCEC2B02D1FFF78DFE45E7EC2B05DC8B
:1043B000E82B00D061E7FFF771FB3DE7F12B02D15D
:1043C000FFF7E6FD38E7F22B00D056E7FFF778FB62
:1043D00032E7F62B02D1FFF707FE2DE7F62B05DCBF
:1043E000F52B00D049E7FFF7A5FC25E7F72B02D115
:1043F000FFF7ACFC20E7F82B00D03EE7FFF72CFBE3
:104400001AE7C046C4070000E0040010F887000067
:1044100010BDC04638B51E4C1E4D1F4B6159E150B2
:10442000231C8C331868FFF7E1F8E26E1B4BA26681
:104430000022E266E2500322605110401D1C022857
:1044400009D090420AD0012802D0FFF7A5FE07E06C
:10445000FFF78AFA04E0FFF705F901E0FFF7B2FA87
:1044600000280CDD6359002B04D1231C8C33196800
:104470000A181A60231C903319680A181A60FA2364
:10448000DB00E258002A01D0013AE25038BDC046B4
:10449000E0040010C4070000CC070000AC070000D7
:1044A000034B0122DA660F229A775A771A77704700
:1044B000E004001070B5084CF425ED006659201C8E
:1044C000064901F0D7F86651FFF7EAFF044A0123D5
:1044D0006366A35470BDC046E0040010D40700001A
:1044E0009C0700007047000030B50D4D049C28600B
:1044F0000C4801600C490A600C4A13600C4B039A8B
:104500001A600C4B0C4A1C60F423DB00D4500B4A9D
:104510000B4B1A600B4B0C4A13600C4A136030BDF6
:104520006803001078030010840300104C0300108F
:104530004403001018000010E0040010654600005D
:104540003C030010E54400007C03001060030010F1
:10455000014B18607047C04648030010094B10B566
:104560001A68191C084B002A03D1084C24682260E1
:1045700003E01A68904200DA101C186001230B60F7
:1045800010BDC04650030010740300104803001013
:10459000034B1B68002B01D1024A13607047C046D1
:1045A0005C030010500300100020704770B5194DD7
:1045B0002B1C98331B68002B04D0174B1C6801235D
:1045C0001C4002E02B1C94331C68F523DB00EB58E5
:1045D0009C4203D1114AAA58002A19D0002C02D1BA
:1045E000002B0BD114E00E4B0C4E1B68002B02D09D
:1045F000201CA95998470023AB5106E0084B1B68C3
:10460000002B02D0201C211C9847F523DB00EC5026
:1046100070BDC046E004001058030010A40700005D
:1046200068030010084B1860084B196000280AD076
:10463000074A01231370074A00211170064A0749EF
:104640008850074A13707047640300106C03001011
:104650008003001054030010B4070000E0040010B1
:10466000400300102D4B73B51A682D4B1168186864
:1046700081421BD000210091019112681A60294BE0
:104680001B688B4202D0684601A99847264B0099C7
:104690001C68181C019A254BA14202D11C68A24239
:1046A00002D0234C0125257001601A60214D224B58
:1046B000EB58002B10D01E490023CB56002B2CD0DA
:1046C0001E4B00229A56012A27D100220A701C494B
:1046D0000A7002221A7020E0134B184C1868002848
:1046E00007D00023E356002B03D1104B1968FFF7C6
:1046F00099FF0023E356124E022B04D1114A0023E6
:104700003370AB5023700023E356002B02D00A20F5
:10471000FFF724FF0023F356EB6673BD4C03001034
:104720001400001078030010640300106C030010E4
:1047300054030010E0040010BC0700004003001008
:1047400080030010B407000038B5064CF823DB00E6
:10475000E358002B05D1E56E034AA350FFF782FF13
:10476000E56638BDE0040010BC07000008B5084A43
:10477000084B126819688A1A05D5FA2252001A6085
:10478000054B1A6801321A60FFF710FF08BDC046DA
:10479000440300101C0000105803001037B5041C1F
:1047A0000025002300930193124B1B68002B02D0BD
:1047B000684601A9984700980135002800D00025D7
:1047C0000220FBF7EBFD0C4B1A680C4B11681868C4
:1047D00081420AD012681A60FFF7C8FF002C04D08B
:1047E000013C002C01D1201C02E0032DD9DD012069
:1047F0003EBDC046780300104C030010700300104B
:10480000F7B5634CF722D200A150221C9432614BC1
:104810001268051C0E1CE050002A0FD118280BD17D
:10482000C32909D15C4B1B680F2B05D1201C3830E4
:104830000E21162200F0DCF8FFF732FEF623DB0033
:10484000002D02D00A22E25000E0E550281C311C65
:10485000FFF7E8FE514E524F336800251B683B605E
:10486000FFF796FE01231E20236701904D4B1B6826
:10487000002B1AD04C4E3368002B16D01B68002B2F
:1048800005D14A4B1B689847474A1368F6E73368D7
:104890001A68013A1A60464A1368002B05DD013B8D
:1048A0001360002B01D1FFF773FEFFF7B3FD002863
:1048B00009DA231C8C331A6801321A60231C9033E6
:1048C0001A6801321A603B4B3B4E9D420CD040238C
:1048D0002A1C9A43394B9A4206D0394B9D4203D049
:1048E000F3239B009D4211D1A359364A93420AD02B
:1048F0002022191C9143344A914204D04022934310
:10490000324A934202D10A20FFF728FEA559261CFD
:104910008C3633682E4A934203D02E4A93420ED0EF
:1049200015E0FFF743FEFBF769FD2B4B1860194BB1
:10493000E0503B68013B3B60284B336007E0284B6D
:104940001B68002B03D0274A0120A1589847019EDD
:104950000198013E002813DC234B1E261B68984754
:104960000E4B1A68214B11681868814208D01268F2
:104970001A60FFF7E9FEFFF7F9FE0C4B1B6898473A
:10498000226F002A01D0019670E7FFF70FFEF7BDF6
:10499000E0040010B4070000180000104C030010E1
:1049A0001400001050030010480300107C03001096
:1049B000740300106E020000C4070000260200000D
:1049C0007A020000FB030000CB030000A3030000F9
:1049D0006A0C0000FA130000640300106F0C000062
:1049E00068030010A40700006003001070030010AB
:1049F00070B5002A10DD047801231C404B1E002BEB
:104A000008DBC55CE4006E083443C4540124013B58
:104A10002C40F4E7013AECE770BD30B59A4205DC72
:104A2000845C8D5C85548C540132F7E730BDF0B561
:104A3000069E051C07A804783078002A17D0059E2A
:104A4000B34217DCCE5CD75CF7193F180020A742B1
:104A500001DB3F1B0120EF540133F0E7CA5C121861
:104A60000020A24201DB121B0120EA540133059A07
:104A70009342F3DD01231840069B1870F0BDF7B593
:104A80000AAC2478099D0094089E2C78002833D025
:104A900000292ED0002A1CD0B3424EDCCF5CD55C5E
:104AA0007F1B3F1B0024A74204DA009C3F190F2400
:104AB00027400124C7540133EEE7CA5C121B0024CF
:104AC000551C04D1009C0F22013C22400124C254F9
:104AD0000133B342F1DD30E0D15C4942091B0024CF
:104AE000A14204D0009F0F24C91921400124C154C0
:104AF0000133B342F0DD20E0002914D0002A08D0B1
:104B0000B3421ADCCD5CD05C0133281A041BE40FDD
:104B1000F6E7B34211DCCA5C0133141B0134624274
:104B20005441E4B2F5E7B34207DCD15C01334942BA
:104B30000C1B611E8C41E4B2F5E701231C40099B6C
:104B40001C70F7BD70B5049C0125257000290BD0A1
:104B50009A420BDC865C8D5CAE4209D10132F7E7EC
:104B6000815C002904D101329A42F9DD00232370CF
:104B700070BD914204DA43185B7843540131F8E781
:104B80000023435470478A4205DD8318013B1B789C
:104B90008354013AF7E7002383547047F7B5134A6B
:104BA000134C13785278C35C134000D04023114952
:104BB00023601231009100220023A6187360009B2D
:104BC0000125123B1F785978C75D394202D07768BA
:104BD0002F437760009F02336D00BB42F2D1123346
:104BE00004320093282AE7D10020FEBD0C010010FA
:104BF0004C0E001058000010122330B54B43334ABE
:104C00000131D318052251431A785C78825C144232
:104C100004D02F4A5F245218947054709A78DC782C
:104C2000825C144204D02A4A7C24521853321470F5
:104C30001A795C79825C144204D0254A7C2452188B
:104C4000A33214709A79DC79825C144207D0204C2C
:104C50005F226418251CA235A1342A7022701A7AAA
:104C60005C7A825C144204D0194A7C245218A03227
:104C700014709A7ADC7A825C144204D0144A7C2440
:104C80005218503214701A7B5C7B825C144207D03D
:104C90000F4C5F226418251C523551342A70227043
:104CA0009A7BDC7B825C144204D0094A2E24521881
:104CB000A43214701A7C5B7C825C134204D0044BD7
:104CC0005918F43127230B70002030BD5800001014
:104CD000B80C0010F8B52E4D061C00272C1C281C03
:104CE00020214F22FEF766F8002F04D02A1C7C23D7
:104CF00039322B7013702B1C4F33002201371A707E
:104D00005035052FEBD1211C2D2338310B70211C80
:104D100037310B70A121A370637049005F23635486
:104D20004221FF316354A32149006254194A11788A
:104D30005278715C0A4204D0221C533252341370F0
:104D400023700024211C301C0134FFF755FF0A2C6E
:104D5000F8D10024104B114DE25C1B19B15C58785E
:104D60000F4A6300084201D0D15805E0D058FEF741
:104D700044F80C49091A0A31281C023400F084FC5A
:104D8000122CE7D1281C084900F07EFC0520F8BD54
:104D9000B80C00100C01001020000010F80D0010DD
:104DA000340000100E01001008880000034B0020A2
:104DB000185642425041C0B2187070478803001024
:104DC000F0B5884C87B0216803900191FCF7B8FBDF
:104DD000854B86481B7886495BB2864A002B07D0F4
:104DE00002235B42036006230B6001235B4202E067
:104DF000092505600B6013607F4B181CDE30458869
:104E000006887E482D04354385421BD1E33358780C
:104E10001D78000228439D78DB782D041B0628436B
:104E20001843774B98420DD1764C0A682368764830
:104E3000033323600921754BFCF770FC2368033BA7
:104E4000236095E22368052B05D0062B09D0042B9F
:104E50000AD06E4A09E001235B4213606C4B029357
:104E600004E06C49029101E06B4A029200236B4D11
:104E7000009300990C244C43002900D10124594B84
:104E80001868022800DCCFE0002305AA53702B68C5
:104E90007F210B405B2B71D02CDC232B00D19EE0BB
:104EA00014DC062B53D006DC002B4ED0022B00D096
:104EB000B6E0492394E01C2B00D18EE0212B00D1D9
:104EC00086E0072B00D0ABE0372283E0402B6DD08B
:104ED00007DC392B6ED03F2B66D0382B00D09FE0FB
:104EE00072E0502B74D0542B79D04F2B00D097E028
:104EF00033226FE0732B69D014DC662B40D008DCC2
:104F00005E2B59D0622B68D05C2B00D088E04F22FA
:104F100060E06F2B3AD0712B52D06D2B00D07FE028
:104F2000352257E0792B49D007DC762B4AD0772BF6
:104F30003ED0742B74D148224CE07D2B22D07F2BA5
:104F400022D07C2B6CD1422244E0202348E0312344
:104F50001370009A022A00DC20E22B1C083B1B681D
:104F60000B40542B30D0032A00D117E22B1C0C3BF2
:104F70001B681940542900D010E225E032232FE0AD
:104F800034232DE036232BE0382329E03923137016
:104F9000009B062B00DC01E22B1F1B6847221940F7
:104FA000232900D0FAE115E0302319E02D2317E082
:104FB000412315E0432313E0442311E045230FE090
:104FC00046230DE048230BE04C2203E0502307E08A
:104FD000522305E005AB1A70E0E1552300E04E23B3
:104FE0001370DBE11C01001088030010780E001024
:104FF000B40C0010480E0010E00400103D001D111C
:1050000011444C8004000010108800003466000039
:10501000246600002C660000146600004C0E001090
:105020000438414241410191019B012B00D184E0B0
:10503000022B00D1F7E0002B00D06EE1296801239C
:10504000194206D0CC4AA01C1178C0B20522FCF748
:10505000EFFA2A68920709D5C74BE01D1968C0B25C
:105060000131C9B201220323FCF7E2FA29680423C3
:10507000194208D0C04AE01D1168C0B20531C9B25A
:105080000122FCF7D5FA2A68120709D5BA4BA01CF1
:105090001968C0B20931C9B205220123FCF7C8FA68
:1050A0002B68DB0609D5B44B601C1968C0B205310A
:1050B000C9B201220423FCF7BBFA2968890609D585
:1050C000AD4B601C1968C0B20131C9B20122032383
:1050D000FCF7AEFA2A68520609D5A74BA01C19683E
:1050E000C0B20431C9B205220123FCF7A1FA2B6832
:1050F000D90516D5A04FA14E3A683368E4B2D1184D
:10510000201C09300A31C0B2C9B2FCF77DFA3968F7
:1051100033680A34C9180931E0B2C9B2FCF774FA2D
:10512000FBE0190600D4F8E0934B09341968E0B2AB
:105130000931C9B202220123EDE02A68019B1A421B
:1051400010D08D4EE7B2B81CC0B231780522FCF702
:105150006FFA316803370131F8B2C9B20322019BFB
:10516000FCF766FA29680222114208D0824BA01D82
:105170001968C0B20131C9B20323FCF759FA2A6891
:1051800004231A4208D07C4AA01D1168C0B2053120
:10519000C9B20222FCF74CFA2B681B0713D5764ED6
:1051A000E7B23168B81C0931C0B2C9B20522012387
:1051B000FCF73EFA316803370831F8B2C9B203226E
:1051C0000123FCF735FA2968C90609D56A4B601C2A
:1051D0001968C0B20531C9B202220423FCF728FACB
:1051E0002A68920609D5644B601C1968C0B2013167
:1051F000C9B202220323FCF71BFA2B685B0667D5B2
:105200005D4EE7B23168B81C0431C0B2C9B20522A4
:105210000123FCF70DFA316803370531F8B2C9B242
:105220000322012352E02A68D20707D5524B601CA3
:105230001978C0B20722019BFCF7FAF92B68022209
:10524000134206D04C4BA01D1978C0B20623FCF7C0
:10525000EFF92968490709D5474BA01D1968C0B265
:105260000431C9B202220623FCF7E2F92A681207C8
:1052700009D5414B601C1968C0B20831C9B2072278
:105280000223FCF7D5F92B68DB0609D53A4B601CE5
:105290001968C0B20431C9B202220623FCF7C8F96A
:1052A0002968890607D5344B601C1978C0B20222E0
:1052B0000623FCF7BDF92A68520609D52E4B601C5F
:1052C0001968C0B20431C9B207220223FCF7B0F951
:1052D0002B68D90515D5284F284E3A683368E4B2B3
:1052E000D118201C02220A300831C0B2C9B2131CE6
:1052F000FCF79EF9396833680934C918E0B20931FE
:1053000006E0190609D51C4B09341968E0B20831CA
:105310000222C9B2131CFCF78BF9009A0435013242
:1053200000920B2A00D0A4E5154B1B68002B06D079
:10533000144B15481A680021144BFCF7EFF9144D73
:1053400000240235AB1E1A7803996B1E8A5C1B7809
:10535000134209D00F4BA200D0580F4BE15C094B10
:105360001A680A4BFCF7DAF901340235092CE9D145
:10537000FCF7F0F807B0F0BDB40C0010480E0010B8
:1053800054010010780E00101F8800001C660000F9
:105390002000001020010010768800000C4E029BB7
:1053A00005A8211C3268FCF7B9F92B68DA0506D587
:1053B000084B32681B68E11DD218074804E01A0642
:1053C000ABD532680548E11D029BFCF7A7F9A4E7BD
:1053D000B40C0010480E00101D8800000867000083
:1053E00038B5FFF7E1F80624002805D1FCF7B2F83C
:1053F00038BD01340E2CF9DC0321201C00F0D8F854
:105400000321C5B2201C00F029F9281CC9B2FCF701
:10541000FBF8092CEDD10B24EEE7000038B5041C95
:10542000FFF7BCFB201CFFF7CBFC094B1B78002BC4
:105430000DD0201CFFF74EFC064CC8235B00E5187E
:10544000211C05485034FDF77BFCAC42F8D138BD37
:1054500095030010B80C00103F58000000B589B04B
:1054600000280ED0FCF737F801A80921FEF7D0F884
:10547000684612300A21FEF7CBF801A8FFF7CEFFED
:1054800008E0FCF730F8044B1B78002B02D00348EF
:10549000FDF756FC09B000BD9503001021880000FF
:1054A000FEE7FEE708B500230B4A0C499A188A422A
:1054B00004D20B49C95C01331170F5E7094B0A4A64
:1054C000591C013B934203D200221A700B1CF6E7D1
:1054D000FBF75CFCFEE7C046000000104401001032
:1054E0007F880000450100107C0E001002B4714658
:1054F00049084900095C49008E4402BC7047C04617
:1055000003B47146490840004900095A49008E44D5
:1055100003BC7047002934D00123002210B4884214
:105520002CD301242407A14204D2814202D20901D2
:105530001B01F8E7E400A14204D2814202D24900F3
:105540005B00F8E7884201D3401A1A434C08A04296
:1055500002D3001B5C0822438C08A04202D3001B2C
:105560009C082243CC08A04202D3001BDC08224343
:10557000002803D01B0901D00909E3E7101C10BC67
:105580007047002801D00020C04307B4024802A1A0
:105590004018029003BDC046D90000000029F0D099
:1055A00003B5FFF7B9FF0EBC4243891A1847C0463E
:1055B000002941D010B4041C4C40A4460123002211
:1055C000002900D54942002800D5404288422CD30A
:1055D00001242407A14204D2814202D209011B0105
:1055E000F8E7E400A14204D2814202D249005B0004
:1055F000F8E7884201D3401A1A434C08A04202D36C
:10560000001B5C0822438C08A04202D3001B9C08AC
:105610002243CC08A04202D3001BDC08224300280E
:1056200003D01B0901D00909E3E7101C6446002CD4
:1056300000D5404210BC7047002806D003DB002094
:10564000C043400801E08020000607B4024802A1E0
:105650004018029003BDC046190000000029EBD09D
:1056600003B5FFF7A7FF0EBC4243891A1847C0468F
:105670007047C04642180023002903D00370013050
:105680009042FBD17047C04670B5061CB30717D1D6
:1056900033680F480F4D1A189A43301C2A420FD115
:1056A000043002680A4BD41894432C4208D10430C9
:1056B0000268074BD41894432C42F1D000E001302B
:1056C0000278002AFBD1FDF7A1FB301C70BDC0465B
:1056D000FFFEFEFE808080805B40253032782530E2
:1056E00032785D0D0A0025732025730D0A00444DA4
:1056F00031360053455249414C20434F4E534F4C95
:1057000045007265616479000D0A4279652E2E2E7E
:105710000D0A004E4F00203F0025732025732020E6
:1057200025694D485A0056333200202025692E2520
:1057300030336956002025735254432000524541AE
:10574000445920464F5220464C415348494E470049
:10575000444D3431204F4B00424144204B455920A9
:105760002530327800202D2025303278004C4344FB
:105770003A25303269202D20256900505245535377
:1057800020454E54455220544F2053415645005316
:10579000574953534D4943524F53202843292032F0
:1057A0003031302D323032310053495A453A256973
:1057B00020555345443A256920465245453A2569C6
:1057C00000535441434B3A0025633120484F555212
:1057D000002D005254432052454144204641494C3B
:1057E000007475726E6564206F6E003C52455345BF
:1057F000543E0D0A00426164206E756D6265722E22
:105800000D0A004241543A2025696D560D0A000DDB
:105810000A2530327820200057616974696E67204C
:10582000666F7220646174612E2E2E0D0A00426133
:1058300064206D6F64656C0D0A00526561642025FB
:10584000730D0A004641494C4544006F6666004CA2
:1058500043442064656275672025730D0A004B423E
:1058600044206F75747075742025730D0A00436FA2
:105870006E736F6C652074696D656F7574207365E8
:105880007420746F202569206D696E757465730DC1
:105890000A006F6E650074776F0053617920626F44
:1058A0006F746C6F61646572202573206D6F726513
:1058B0002074696D652573202E2E2E0D0A004C6113
:1058C000756E6368696E6720626F6F746C6F616478
:1058D0006572202E2E2E0D0A00000000005C000CC8
:1058E000000C7C287C7C447C241048285408000C44
:1058F0000038440044380020100810381080400060
:10590000101010004000201008384438007C00645B
:1059100054484454281C107C4C542438542004749B
:105920000C28542808543800500080500010284497
:10593000282828442810045408384C5C7814787CB3
:1059400054283844447C44387C54447C14043844FF
:10595000347C107C007C0020403C7C106C7C4040FF
:105960007C087C7C047C7C447C7C14083844787CF7
:105970001468485424047C047C407C3C403C7C20DB
:105980007C6C106C1C601C64544C7C44000810201F
:10599000447C000804088080800408007844780073
:1059A000040603000000007F010704000007000058
:1059B00000070B064400FF0144004400FF014409B6
:1059C000058C009200FF019200620C0686004600E2
:1059D00020001000880184010C06EE001101110165
:1059E0002E01C0006001050300000000070905004A
:1059F000000000010182007C080400007C0082009D
:105A00000101090510005400380054001009051068
:105A10000010007C001000100603000080058003C9
:105A20000B061000100010001000100010060300FC
:105A3000008001800109050000C00030000C000357
:105A40000B06FE000101010101010101FE0C06002F
:105A50000004010201FF01000100010C0682014166
:105A6000012101210111010E010B0682000101112A
:105A70000111011101EE0B06300028002400220064
:105A8000FF01200B068F000901090109010901F13D
:105A90000B06FC001201110111011101E00B0601BE
:105AA000000100E10111000900070B06EE001101E1
:105AB000110111011101EE0B060E0011011101116E
:105AC0000191007E06030000980198010603000082
:105AD000980598030A05100028004400820001017F
:105AE0000B062800280028002800280028090501A6
:105AF0000182004400280010090502000100610134
:105B000011000E0B06FE000101190125012901BE3D
:105B10000C06FE011100110011001100FE010B0620
:105B2000FF011101110111011101EE0B06FE00012F
:105B300001010101010101820B06FF0101010101C7
:105B400001010101FE0C06FF0111011101110111FA
:105B50000101010B06FF01110011001100110001EC
:105B60000B06FE000101010111011101F20C06FFFB
:105B7000011000100010001000FF010A05010101D2
:105B800001FF01010101010B06800000010001007D
:105B9000010001FF0C06FF011000280044008200F4
:105BA00001010C06FF0100010001000100010001DC
:105BB0000C06FF010400180018000400FF010C0689
:105BC000FF010400080010002000FF010B06FE008A
:105BD0000101010101010101FE0B06FF011100118C
:105BE00000110011000E0C06FE000101010141012F
:105BF00081007E010C06FF0111003100510091006F
:105C00000E010B068E001101110111011101E209B3
:105C10000501000100FF010100010B06FF0000016A
:105C2000000100010001FF0B061F006000800180E1
:105C30000160001F0C06FF014000300030004000F2
:105C4000FF010C06C3012400180018002400C30142
:105C5000090507000800F0010800070C06C1012132
:105C600001110109010501030100070804000000FA
:105C700000BF01BF0109050000070007000700077A
:105C8000130A00002000E400FC003F00E700FC00D5
:105C90003F002700040F0800000C011E01FF03FF56
:105CA000032201E201C2190D00000E001F001101C4
:105CB0009101FF007E00FC00FE0113011101F001C3
:105CC000E0140A0000EE00FF0111011101BF01EE16
:105CD00000E00130011001050300000F000F0A056C
:105CE0000000F800FE03070701040B060000000097
:105CF00001040707FE03F80F08000000000A000E69
:105D0000001F001F000E000A110900001000100003
:105D10001000FE00FE00100010001008040000003B
:105D200004800780030D0700001000100010001011
:105D300000100010080400000000800180010D0721
:105D4000000C000FC003F0003C000F00030F080020
:105D500000FE00FF01010101010101FF01FE100829
:105D60000000000002010201FF01FF01000100012B
:105D7000100800008601C7016101210131011F01E6
:105D80000E010F08000082008301110111011101B1
:105D9000FF01EE11090000300038002C002600FF42
:105DA00001FF012000200F08000080009F011F015B
:105DB00011011101F101E10F080000FC00FE010BCF
:105DC0000109010901F901F00F08000001000100BB
:105DD000C101F1013D000F00030F080000EE00FFBC
:105DE00001110111011101FF01EE0F0800001E0059
:105DF0003F0121012101A101FF007E0804000000F4
:105E0000008C018C010804000000048C078C031234
:105E1000090000200070005000D80088008C0104A8
:105E200001040111090000480048004800480048EA
:105E300000480048004811090000040104018C01D9
:105E40008800D80050007000200D070000020003F9
:105E500000B101B9010F0006190D0000F800FC01A6
:105E60000603FB06FD0505050505FD05FF05060105
:105E7000FC01F8120900008001F0017C004F004F86
:105E8000007C00F00180010F080000FF01FF0111FC
:105E90000111011F01FE01E0110900007C00FE005C
:105EA000830101010101010183018211090000FF49
:105EB00001FF010101010101018301FE007C1008C5
:105EC0000000FF01FF011101110111011101110178
:105ED0000F080000FF01FF01110011001100110067
:105EE00001120900007C00FE008301010121012153
:105EF00001E301E20112090000FF01FF011000109F
:105F00000010001000FF01FF010A0500000101FF61
:105F100001FF0101010B060001000101010101FF68
:105F200001FF10080000FF01FF0138006C00C600EF
:105F30008301010110080000FF01FF0100010001C1
:105F4000000100010001160B0000FF01FF010F001E
:105F50003C00F000F0003C000F00FF01FF011209BF
:105F60000000FF01FF010F001C007000E001FF01B5
:105F7000FF01130A00007C00FE0083010101010102
:105F800001018301FE007C0F080000FF01FF0121D9
:105F900000210021003F001E140A00007C00FE00CA
:105FA00083010101010101038307FE047C0412093E
:105FB0000000FF01FF01210021007100DF008E01C0
:105FC0000001110900008E009F0111011101110152
:105FD0001101F301E211090000010001000100FFBD
:105FE00001FF010100010001110900007F00FF0015
:105FF0008001000100018001FF007F1109000007FE
:10600000001F007800E001E00178001F0007190D73
:1060100000000F007F00F001E0017C001F001F0066
:106020007C00E001F0017F000F120900008301C72E
:10603000016C00380038006C00C7018301110900B1
:1060400000010007001E00F801F8011E0007000112
:10605000120900008101C1016101310119010D0125
:106060000701030100040603000000007F0107048C
:10607000000007000000070B064400FF0144004435
:1060800000FF014409058C009200FF019200620CA0
:10609000068600460020001000880184010C06EEF0
:1060A00000110111012E01C0006001050300000074
:1060B0000007090500000000010182007C080400BF
:1060C000007C0082000101090510005400380054D2
:1060D00000100905100010007C00100010060300DD
:1060E00000800580030B0610001000100010001047
:1060F0000010060300008001800109050000C000B7
:1061000030000C00030B06FE0021011101090105FE
:1061100001FE0C06000004010201FF010001000164
:106120000C06820141012101210111010E010B0622
:1061300082000101110111011101EE0B063000284E
:106140000024002200FF01200B068F000901090135
:1061500009010901F10B06FC0012011101110111E5
:1061600001E00B0601000100E10111000900070B2D
:1061700006EE001101110111011101EE0B060E00D6
:1061800011011101110191007E0603000098019890
:106190000106030000980598030A05100028004432
:1061A00000820001010B0628002800280028002892
:1061B0000028090501018200440028001009050299
:1061C000000100610111000E0B06FE000101190122
:1061D00025012901BE0C06FE01110011001100115C
:1061E00000FE010B06FF011101110111011101EE69
:1061F0000B06FE000101010101010101820B06FFF6
:10620000010101010101010101FE0C06FF01110163
:1062100011011101110101010B06FF011100110013
:1062200011001100010B06FE000101010111011115
:1062300001F20C06FF011000100010001000FF0119
:106240000A0501010101FF01010101010B068000A6
:106250000001000100010001FF0C06FF01100028F1
:10626000004400820001010C06FF01000100010052
:1062700001000100010C06FF0104001800180004D1
:1062800000FF010C06FF010400080010002000FFC1
:10629000010B06FE000101010101010101FE0B06D7
:1062A000FF0111001100110011000E0C06FE00018B
:1062B000010101410181007E010C06FF0111003145
:1062C00000510091000E010B068E00110111011109
:1062D000011101E2090501000100FF010100010BAC
:1062E00006FF000001000100010001FF0B061F0076
:1062F00060008001800160001F0C06FF014000303B
:106300000030004000FF010C06C3012400180018F3
:10631000002400C301090507000800F00108000778
:106320000C06C1012101110109010501030100044D
:10633000040200007F0109050000070000000000C2
:10634000070B064400FF0144004400FF01440B0614
:1063500000008C001201FF032201C40D07820045DA
:10636000002500920048014401820C060000E6006E
:1063700019012601C00020010704000000000100EF
:1063800002080400000000FE0101020804000000F1
:10639000000102FE010B06000088005000200050A2
:1063A00000880B06000020002000F80020002006D6
:1063B000030000000400020B060000200020002063
:1063C0000020002006030000000000010905000075
:1063D000800160001800060B060000FE00010101AC
:1063E000010101FE0804000002000200FF010C068A
:1063F000000082014101210111010E010B06000084
:106400008200010111011101EE0B0600006000582D
:10641000004600FF01400B0600009F000901090132
:106420000901F10B060000FE00110111011101E24A
:106430000B0600000100C10131000D00030B060036
:1064400000EE00110111011101EE0B0600008E009B
:10645000110111011101FE0804000000008C018CE3
:1064600001080400000000000208010A05000020E5
:10647000005000880004010B06000050005000503E
:106480000050005009050000040188005000200B56
:1064900006000002000100610111000E0D077800E6
:1064A000860132014902390242027C0E07800170E6
:1064B000004C0043004C00700080010B060000FF00
:1064C00001110111011101EE0B06FE000101010194
:1064D00001010101820B06FF01010101010101829D
:1064E000007C0C060000FF011101110111010101E6
:1064F0000B060000FF01110011001100010C06FE47
:10650000000101010111019100F2010C06FF0110CF
:1065100000100010001000FF01080400000000003F
:1065200000FF010704C00000010001FF0E0700008A
:10653000FF01180024004200810000010C06000049
:10654000FF0100010001000100010E07FF010C0026
:106550003000C00030000C00FF010C06FF010600F7
:1065600018002000C000FF010B06FE000101010120
:1065700001010101FE0B06FF0111001100110011C4
:10658000000E0C06FE000101010141018101FE0225
:106590000C06FF011100110011002900C6010B06B5
:1065A00000008E00110111011101E20B0600000133
:1065B000000100FF010100010B06FF0000010001C6
:1065C00000010001FF0D0703001C00600080016056
:1065D000001C00030D071F00600080017C0080018B
:1065E00060001F0E078301440028001000280044AB
:1065F0000083010D07030004000800F001080004F7
:1066000000030E078101410121011101090105016A
:1066100003010000060B205A64600000030720619C
:10662000D95800000D0C205A2E6300000D0C205A82
:10663000695C0000060B205A9F5900000007000803
:10664000000A01001811101338313033787170735B
:10665000C8C1C0C38881808384848782C5C4C7C2FF
:106660007574777235343732151417120207020821
:1066700002010003010903040204020503050006E8
:106680002024282C383C4044484C4669726D776180
:1066900072652025735F5633320D0A00252D313087
:1066A000732025732573000D0A5479706520273CEB
:1066B000636F6D6D616E643E203F2720666F7220B0
:1066C000706172616D730D0A0025730D0A0D0A0069
:1066D000564F5941474552203E3E20002563004811
:1066E000656C70004E6F20706172616D73004B6558
:1066F00079207072657373003C6B6579313E203C84
:106700006B6579323E202E2E2E0044756D70206D03
:10671000656D6F7279004C6F6164206D656D6F728D
:106720007900637400436F6E736F6C652074696DDC
:10673000656F7574003C6D696E757465733E0062BB
:106740006F6F746C6F6164657200496E766F6B6514
:1067500020426F6F746C6F616465720053617920C1
:1067600074687265652074696D657300476574208F
:1067700074696D65007473005365742074696D6588
:10678000003C595959594D4D44443E203C48484DD0
:106790004D53533E007464005570646174652074F9
:1067A000696D65003C6F66667365745F696E5F6DE9
:1067B000696E757465733E006B6200546F67676C39
:1067C00065206B6579626F617264206F7574707596
:1067D0007420746F20636F6E736F6C6500546F6705
:1067E000676C6520646973706C6179206F75747073
:1067F000757420746F20636F6E736F6C65005265E3
:106800006164206261747465727920766F6C746162
:10681000676500001757000000000000651E0000BB
:10682000DF660000E4660000E2660000FF00000092
:10683000A1120000EE660000F8660000B9690000D1
:1068400000000000C51000000A670000E4660000B8
:106850004769000000000000651100001667000095
:10686000E4660000226700000100000051130000F0
:1068700025670000356700003F670000000000004A
:106880008D1300004A6700005C670000236700006A
:1068900000000000ED0F00006C670000E4660000DF
:1068A00075670000020000004D10000078670000CE
:1068B0008167000095670000010000008D10000056
:1068C00098670000A4670000B8670000000000009F
:1068D00025130000BB670000E46600009667000017
:1068E00000000000F9120000DD670000E46600000F
:1068F000B967000000000000D90F0000FE6700002B
:10690000E4660000008001500080025000800350C7
:10691000FC3F0150FC3F0250FC3F03502578000D26
:106920000A413A2000202025633A20000D0A533AFC
:1069300020000D0A4D3A20002020473A2025303211
:10694000780D0A006661696C00253034692D2530A8
:1069500032692D2530326920253032693A253032AE
:10696000693A2530326920257300253032783A257E
:106970003032783A253032692E25303269002530A0
:106980003278203A202569202569203A20253032A6
:1069900078004E4F2052544300253032783A25304B
:1069A00032783A2530327800253034782D2530324F
:1069B000782D25303278202025730000DC69000016
:1069C000E0690000E4690000E8690000EC6900008B
:1069D000F0690000F4690000CF6600004D4F4E00E2
:1069E0005455450057454400544855004652490007
:1069F0005341540053554E00CCC5ED65B706894749
:106A000017C5304D1D8E212B182C0A4A20F8B9A22B
:106A1000F0094F3B9688E439683B3EA814CE4D55AB
:106A20009FCF2C009D2A121B0BD5FEB55BBF6D813D
:106A3000F26D37363CB4F43E2F2362A699AC8A0A35
:106A4000E7B91698B086BC0C7E32A93A254743991F
:106A5000F4214C090934959BC825BB24186029CD25
:106A60003565F5C7CC3D459C153300BCC38D1C076F
:106A7000AAEE182B886BAC34BE74E471824DE71615
:106A800035C45D87238AF03B53D61F67A85ACA0BCB
:106A9000160ADDBC05B5002A40A8E540E4D9020687
:106AA0002F23711CC078F30FA1E765D0C64D24F8E1
:106AB000513F30813CA8B2493B07D2ADF259C510D5
:106AC000BEBF03B9DF0FAF81CE475EFD58BBCDFD22
:106AD00055E21E4DD181D86E557EE9F09504406D8A
:106AE000A0809FEE4160222DB1C51AC524A7B937F9
:106AF0006F7B57357F482334EB41170218793402F6
:106B00007A351A00007FBC9D7E59BE6F5DCC9D50CA
:106B1000D6C9465756E7C3E4D2A85C21B5B6E648C5
:106B20004CDC2130433E5CAEF4F924A7A411CAFF2B
:106B30000D0F20FE12DA997EAD1BBF116F6618C5CE
:106B40001A9A9CC93A5C34173F2125E2555DCE83E1
:106B500043B3D5D80AA88D812D4F9B9EB019B15D46
:106B6000F9FD426B3B60AC8C65ED496F0BB8CB0E09
:106B7000923C245807E7766BC5428D4B5CC3BFAD92
:106B8000E1A0DD080EF360CAFDF268C38AD5D14AE0
:106B90007E0E2A977950C7996878594B4A70170E1C
:106BA000DCF1B888CFB91429E358A3D1F15BD151F6
:106BB0006A559385F6AEC0327D06BB82994D4D89EC
:106BC00061DD6E7B87C01F058779201F4EEABB9170
:106BD000C8F3A88DA1E70610883D2E9FD53B0F4531
:106BE0002323BDCA32002D1EC2487AC1C11B6FF5D6
:106BF0002AC3BEBDB44BB5A3BD1CDBD5E7D04DB891
:106C00007F213EB756392FD448532A66739478486B
:106C10003EC9F2DAFCDA4B99E0BCEF88A177A8AA6A
:106C20007060F7FBC4FC73E214B55A92999C238CF4
:106C3000381614AD641AE23B87D3636733ABC205E1
:106C40009C29DEA81EC8506A921AFCADF9AA2C4AEB
:106C5000605408AFF93B12894E9339FE0D58BB873B
:106C60004DEDD8AA6DC8D3D6D0B17B624D1EF45A73
:106C700082D405BEAFF4352670CB25C836391C77D3
:106C80001FD558090F6F8F6C644B5ECCA4CAC08CA3
:106C90001B678FF7A6493D49FA5226C5F103CBD1B0
:106CA000C09E334657A63B53B68388668CF5BCC45A
:106CB00092859C4B4E7BC27581EC71F21E9AB24B51
:106CC000E30ED65DF17F012703C52F639DA73841F1
:106CD000A047D2255A018C48F66087D6EEFC57C0F3
:106CE0004E0525F5DB42A6C16CF92BF1BDF85E47D8
:106CF000FC047B909633B21078BF1229C2230E5247
:106D0000D150D71F37D9C1A778E8B0FEDF03BE4501
:106D10009868897DA17227144DE0370514A15C2B7A
:106D2000756241E20271B6B785069CEE84582874FC
:106D3000AB82E17252C7FEBA2CCBC9E57964D52A81
:106D40000AED5091D7D5FB9B8370951C10CAD4BE19
:106D50009D36C1596052495534EF989004591598A1
:106D6000D0E488071E8B8F4A1894491214388E0776
:106D700019352F563F1AEDA8F11C81EFF519C4FD06
:106D8000108CBAE3283D2513C852E9DC73436DB675
:106D9000EDB7D580363069003D3F6A3EEE4A481B6C
:106DA000E1B7AEFF706515A4B45383C8DEF50B469A
:106DB00065296FA594986D5BBC58646ECA3D9A6D49
:106DC0001A1190F9E8C05D9EA2EFCD8DB9B5E9DA50
:106DD0008FF38037B26C921C5DC0EF64291B9E60FC
:106DE000BB269607EA3B91A386A93722D12D755D74
:106DF000A3C0BC82A89A4F61B30B18F72A7A1BB2C2
:106E0000E3BB6668F246A9F2C172155441F96A30D3
:106E10003BEE635DFC384B3E21B48A65F73D12AF13
:106E200004B68AC46C58A87CD526964D9C9EE9E889
:106E30001E40D89FFC4B15837C239C9EC07F01B2D3
:106E4000F2969B7494A1825813F652BD0901E4C6D0
:106E5000EF28637193B2A8238CE7AD202F52CC2C7E
:106E6000FAFD72C5E739337FF5F68DF5B5A22B171C
:106E70002E0C78723FCB7F3360BE9352E761326D48
:106E80009C09077A0D2DE5DA86EDC32F669758E148
:106E900075C396BBE347DE72DAA43DE9E7A087F449
:106EA0000D7DBB5ADC5F76069AED150290FD2AD562
:106EB00090DFBE9CA29B0A85D4B51EB290AE50E86E
:106EC0002B1066C4F2E34F0AEF68D42616C9FF3BC5
:106ED00075F0908A1D7AF061F048D502B5B4AE34F1
:106EE000F7032D62B6C7A0A52A5C832ECEB988FF12
:106EF000C6BCC428AD834396627F47EF35197EF345
:106F00004B2B5CE5E1B3316D42CC9DCD5C1D678BB5
:106F1000A0D715829D39C0049664C78C63B8DE245F
:106F200061CC01A4F75C15C0B93FEE2D595027790B
:106F30009B3E0D1E6EAA6B4B37780E6EA203292A5C
:106F400041B187BB15A7AE7FAA799C0B2E4165F690
:106F5000FA42B75AE2E312E476FDAA5D6E0D7FEBCA
:106F6000B8DAA3B139D8163A426A746984B5340FD5
:106F70000D1C6789A976D71763166E038DA10BA91F
:106F80005E1CC407E58A67BE815BFD3033A304261F
:106F90001B20F63D2D6AA4726018A3D88398272879
:106FA0009CDCC8AE7064E06A2280A069B11C9B536F
:106FB000DD2677CF410F14D18138399028B91C03D1
:106FC000944980C86EB187DA3EDE2B98AB61841F8E
:106FD0002DC8FAAB0F2874024BFDBEB8FA97832F69
:106FE0007C2F494CFF1CB6E09047483867A1D0730E
:106FF0009D342055FFDBEFF020483786C3EB22E9B4
:10700000C8020F09E0C0AF96AF2560CCE142E92687
:10701000C1D2F3BC847794D09893475D4B0EDF8444
:107020009EAA3380213EB2D101C4B15717FB6F1F16
:107030004C352A23F4EA807A2903D9C38834A6314F
:107040002541EAEECB0BF00F4F2B31C9B54234CBC3
:1070500001C24D520B56D3B1270EEAA496ACB340F1
:1070600052D0609DC5B39BC881B228B2492F1DA9DB
:10707000875EDA9B2503B1222F1A68ACED4BC3095A
:10708000417267449B2C01836A11F92AFD9BBA1453
:10709000205F6191C0BFB5081CFCD7BAB863304F00
:1070A0004BB73AFAB4B9FC890C008275E1F751EF9D
:1070B0006EA4A41A41C38AE13A55C67358EAB80EC1
:1070C000CE007DFB42E6AA8344C1F4EC520003DE0D
:1070D000B2468397F02F755496720DEA485DDFE44F
:1070E0007AA9761B56507F2C2929FD6CD57AE46647
:1070F000BF893B2CFD16CE9AFC218DCEE05D9428F5
:107100001CBBB04BE9E1ED3D65AFC86ADA81272DC4
:10711000D2B6798A1F779C7815CBCFFA5B26F6AF6B
:107120008044B30F434409C6ED140644D980FBC420
:107130005C56689E55DF0656F2C8345D9711A4F57B
:1071400069F70F0E0CA1472CAC8C509A501EDE999B
:107150007B8A87B643EE18CE1315F7847CC09C8BD0
:1071600071CC341C884B65C1B9DDD759E352433526
:10717000ED4D9A0EB5BAD18E9E942C8CA89D1E60B2
:10718000AE2D2CD1B76CC7D4034FE646DCB9BB5348
:10719000F5EAD86F2064EDE74CA734D8E9FA4BBC88
:1071A000E69EC2C26BC4B6B4D3F4205890FF443EEE
:1071B000CB8432332CBFD21F8C1DD12646A58A32F8
:1071C000F4CFD5A2E60088B9912032A8F2D496A4D3
:1071D000BB012FCD3F40E02ED6A81A785DB5928A2C
:1071E00043FA4EE1B472E84DD5201913914AD79F66
:1071F0003D3F63ECA337430A2726EA4A78B4F8995F
:10720000241A1FC033C89D8D593739860A71F9FD7C
:10721000CBD173073E814192DBF63C60CF9A469F0B
:10722000A70FA641C49F98961BF5D45F197D3D1FFB
:10723000D230B6887A62E30D9D15686AE45949D167
:10724000C6E3FA094152E29FB84CDFF455963093F9
:10725000DC02CA1A79D92DE3048B746A30208F833B
:1072600051B342045F92B7B222F49FB86C5D94931D
:107270005C8D2CD7A94B3F7559554862C72F4FB02D
:107280001F011606A9D138EA09BB7A1032266F937E
:107290007675D6764B068175C4E4214739E028110E
:1072A00012F1971B6069EA2F9D0D4CAD4BDCF56820
:1072B000C9A90BDC38D5710790A5DB2341CC0F0F92
:1072C0005177428AEB3A55F86B8DAAFC2848BB549B
:1072D000CB1E1529FF1B9D5A919CEA67C2EA847A4E
:1072E000ECD73F7D5C90C2DF2890CEBDE0CD01EEB3
:1072F00024BE267115A6CEDA82BF73B6AD0304E3B1
:107300008656D1C663B0229E7606CAB926625C66EE
:1073100002CF70AD14BA1C7A711FFF7C6021D801B6
:10732000261B7C350E97784A09D0E2DB438A42213E
:10733000521EBD8DB4ABB8F8756E52B1AA9051799A
:10734000AEEC3A8D09C6009AF46DD1DDE05A396091
:107350008133610227366D6F8C4F299546530404A3
:10736000AA2C1F807C6012D7B6872D050A760D32B5
:10737000303AD08D441B3336E492B29D5699415B2E
:10738000817DD5D3C9AA2EEF0F139C36F99E81E1DA
:10739000524DDB0074A957D3B954524C94F2E3CF49
:1073A000F5173EFFE37DEFCFEF1CDFBF66CE68C56C
:1073B000DCA1C83D6AAD28F45ECD750863A03762D4
:1073C000604C4A5A5B5EC46A0B79186F6A71628DB1
:1073D000C28B2B3AD2B5104DC270FC9F2657DA46AD
:1073E000AD5D9FB9FFD42D02000D066950B87DDC5C
:1073F000A8A3AA50F238E7D2BD02E9CB971165E401
:10740000219449C73984657FF869C1C53244CE44A7
:107410007E072BACE3C83369F42083477EFFFEABC5
:10742000F5F1650BC31212F3CB9B0894932E9E8D3E
:10743000B4DAB7A369446AC4C8B068F66D51697A12
:10744000ED35C203FDD482B20804AA8BDFF0A54655
:10745000902C9B799E845A2A8E000F1D63BCD70303
:10746000642A1C77B6B23E6B85822351C1D9CEBC4B
:10747000366BC9139EDC0A367E17FA006BC570178F
:1074800035E38541EEF556F1B47C1D22F7FB5945F5
:1074900006C9E9F2CD7E92129D461750C371052CA4
:1074A000A40F5C15731980E864E2F3F4B46F925F83
:1074B000E0BC5558C24504016E9C5D0D1BBB8B2181
:1074C0005DACC26A5D435564646F0B25F535589811
:1074D0003E84006EB0D13A283FF140663E09CE208E
:1074E000076593A94E331F1749600A02F4D409DADD
:1074F000EB504E14F33712571244930018D823CF91
:107500001C720C558A188756E5358ED004EEC911C9
:107510000ABF5F48D277B8411C961EE2D7811F7F11
:1075200086D4B5699E7702D04262D98043B21D33BA
:10753000949717BA284B5B4BB46500C89CD9988DBB
:10754000DFD1A530912E24F8E4CD55DE522F6DD633
:107550005D376AA379CBDD750E3D4D73A9251ACF32
:1075600047E3F1165B4C98733951ED82A2E3F99C25
:1075700051BDF56B218661C62303650939F5091EE6
:107580004292DC11100C0B760D1C988DD359784962
:107590003FF1E8ED32F4F0EB0FDF29688936024461
:1075A0000F11D8E5521E550309B20E719887535F2B
:1075B0004DD4E40B91B84CF75D8854F4EBE39BDDBC
:1075C0005AB847BF0C05FE8BD50FC3D1166A422BA4
:1075D0004D6C65696B92750517EEC5CA1E1181F376
:1075E000907C990795373CB811ED3EC65C24E77551
:1075F000EFDFD41494BFD89E2A1FF2A783ADD80919
:1076000073D947B20FCC6F2221AA8EA55AEF857687
:10761000D6914764C047909E7B3DF557D3BCD9298E
:107620001E4FA529A40058C926BCDEC24624D16A33
:107630000C025ABCD1C4162A33E69CE77AE0CBCAC6
:10764000DA59FECB1E10256612C5C406073CEB5D59
:10765000E1EE18515564D10EB1170B865BC4EAC632
:107660000116595D3E6979F4F12EAB639E9B291496
:107670005B96290788DCE868A8732BBBEFCC73B74F
:10768000D4055C9C1D5EDD2A12CC0BDE6B169A07BE
:10769000FAA23C94147A8B3F51B148CC847B97C2B8
:1076A000545312E8D51290E710DD55F74749067E8E
:1076B0002B4BD019A82507F8616AA52ACD6767AAC0
:1076C0003447557F70885F64DD91F78C9B1FD5F53B
:1076D000B091A7AC1DDA9B6A0711C0F72A2D91DE85
:1076E0004B829AEFB537D39DD33BBBBFBF54056EDA
:1076F000DC92618287B9D8E56FD2D228A360B60F39
:10770000F0CE2FF74DB653BD8F275110AD467926D9
:10771000C2E435F0DE52642173D29EA44394909665
:10772000B60158A6F3FCDE904939D85CD54BDD1F75
:10773000229AE2ECDE1509916B468F7267D24CF506
:10774000241DE8AB1A163109E3E16B9EB0DCC5904D
:10775000FD76F239970EAAB237094D13A841B08CC5
:10776000E8E8079DA5F5EBFF9585E687E32488ED1E
:10777000DDC09E5B38D4ACB8AA642AC372A082E292
:107780003E72DF4145033C42167F2B5118E5D2EA99
:10779000BCD7DCDED2E138EBBE56D885DFA7313D61
:1077A00067382122B98DDB684DB0D4F717D559BAA7
:1077B000DEBFDAF6B0DA58EFB671D94DAFB0363A6F
:1077C000DDF23C39004FF2056CBB75BA469D75F68B
:1077D000D581F71221EC232601908BF47D5794DAA2
:1077E00096790CFC564B9AC00EA70A9C42FB3BCFE5
:1077F000A406A8217B722DC76A88467004FEC6A61F
:10780000857117B98D25C2CA7198D6008B0CAB3023
:107810006E9015DC649F18D3AE7329B9F21D161E45
:107820009E4759375C648593447B5B455128DB1147
:10783000593A9B53F2120A7E7DB8EE59CD05401A93
:1078400092B2494531A6FC6C2C6281A8C6DFDF15D7
:107850002BE8864DD6E617C880DD13A10A518DA509
:1078600028D5BA55EAD26506E250FF2F14769C2738
:107870001859E65A310EFADC3720FF642C12EB83DC
:1078800080945DB8269A67C6F98F8958C7A4AAB8AC
:10789000FBA879B66F1457D45754DB2379F00A5BF1
:1078A000B77E09E0C43C2D9EBA4DD0633C919D8FBC
:1078B000122D7C7A7BAB0225443EF462B962E1ED85
:1078C0008CBA3B65CD979FB21348E949B57F5FB34A
:1078D000C074719A89D8CF9A3B6E78BC9AD77F6A68
:1078E00039F229D63069ECF8DC3AE631966826FEA2
:1078F000270061DC72EFA503887C8E98C6E43DE822
:107900001B3085802CB076BBEA1D770E856D37C99C
:10791000D683FE5A414E62585BE84438CB9CC37311
:10792000A25D3DD80D02FEC8718842D36CF1B90743
:10793000A4FD1A64F7114DC2F3F77EAF6A4AF33C17
:10794000921292919BF12EA978218B19BCB53154DA
:107950008516FECBF4622ADEAD47186AB637014FB2
:107960009220C35FB2F4820280C959CD0E13046223
:1079700081D4E3E99A5482CE871B15C88F020C0C80
:1079800067191780633690F80004E4EEA55BC6E43F
:10799000B8C4F86A94E53C7FBDBFB2B3C1F694BBEE
:1079A0000272262BFDFBBB260D8F6BEF2B16CB9E99
:1079B00098FCBA68F35AA947DEA8CB589D54B0A6E4
:1079C000D07618AED0234367BD5F07094230CC653F
:1079D000C1EADA2D1A11167D581CCAE3A1CE3A3736
:1079E00080009B4C9FA973A71670D9EB72911E7EE5
:1079F00076FFFC3D47A2AE61EC32D48095198961D7
:107A00002DF6BB1C55E7DBEDA37945DBA55A080D28
:107A1000CEF92EB701905F5BE14A1793BADABC2228
:107A2000E98FF046C8CB85CEB00335D4C6FBB6C9C6
:107A30003F707E31BBF8AC4BB96F84A540F938F389
:107A40002A8A0C439171A0249D2D7D2736AC63AC0E
:107A500011EF01731F57A0238F78ADF582FE3F15FC
:107A60007C0247D9246AE2B23B096B80223E98FA35
:107A7000A248F1D6985EA57C8134EBF4C66F8C3DAC
:107A80007E3BD9B9F5524505617B6B3CB2778CDE04
:107A9000F9104987ABFC4592D3EA9A7F965C35583A
:107AA000AE5B2662CC4B013AF0A26F6EE0885026A6
:107AB0002A627F7F551D7294C43466D08505EF0E0F
:107AC000626865726266254DC32B0FB32C12D972A2
:107AD000B4A305A1402BF6BE3E9ED0DCFFED0420F2
:107AE00015631F021A31D2DDF9ADC5BB55ACB56DBA
:107AF0006E4D22E063B447D3E089E6723176B883F5
:107B00004B5B918F3B8427BC3C29C73712477D0FC5
:107B1000558EB14C70BEC67C4CAB1DF57E02D4E8D0
:107B200036DC026560D0C10ABC082D391F93D293A0
:107B30008FE32340DD2D8120209410814F4709B72A
:107B4000A61BB6B829A6A912DF3F2A32CEF214F638
:107B50009983F139C854C8D5922DB93B1C146C4D8A
:107B6000B1E9B2F3E93045E876215D8A18411BA0FE
:107B70007541F07660DD19848A5299000561A4CDC3
:107B8000C7CA5FA93F61521B45340D2456100C4AE9
:107B90002624013977094E0892275468E34C6B1369
:107BA0003ECAB4F991F7C1CC40864C40C8F549AE05
:107BB000C50D46B1A6D2AC9098D0E22485CFF39300
:107BC000A5893CBCD4104A7088DBF2263D39C3F746
:107BD0005BD85E6268258A522CEFB85FCC1083B404
:107BE000C3AD9147E45E2D27BB3A62022A4C137C59
:107BF0008691B909957B1BA7F74F2F72335916FB56
:107C0000A3A8B68305C1F5C900E2675C56102D3301
:107C1000C74E8F7D4D39DA97ABDD2FE64CA652FB70
:107C2000D6B49B73BC5F8974018BA1AC588E30BCF9
:107C3000A6ADD72B8E8D9E7E144F60AF0135FE18FA
:107C4000F06DD385B82CE47E7E6AE950D1B7D308B5
:107C50004529F333ACDA98470F18F891F27378E5B9
:107C60009D9184163D188574A7EDCACB03B50D4FC1
:107C70005618D505CD73B5EEB1ABB9377A49B748CB
:107C80002D0CB5EE9060EDCD88837E640C3A35C83E
:107C900039492BA8603ED93C48D883B5A432ABDB28
:107CA00083CE4CF4FAE40710CB6F850C7DF27AE0BA
:107CB0002EB8CE97E02739C34B6CB9464DB28475C8
:107CC000EE8FF0543245DF33A30CC269E91E2F4911
:107CD000269F8AFB7546263C9BDBBDADEA164F8D81
:107CE0006785670F65A6F0BAA3EA9DD81BACE2CF03
:107CF000CD4983BF9E3EB18055996328897B234A35
:107D0000C8C5E97C2A8FCC8D57793FAA1CFFCFDAF2
:107D100089640388F1C8D946C057B969EB445EE964
:107D2000F6E2269578C81E75FFE3D293DF0ABB60A2
:107D3000E2C74F68EC84BE48D1941B11477CF384A2
:107D4000E8FAA845EC5133A27F99CD41F07E2A1084
:107D50000175B4D5C25B215F2917B706111A8D9141
:107D6000A57DEA6A97377F41C5B81508799E5061AD
:107D7000EA2F0543FC3400B8B6EE75B1926999015B
:107D800021285BF7843BAC5FB1B55B57CB69EAA8B0
:107D90008C0576320EEDDACE4E485B3DCF99A8DFEA
:107DA000B81EAB419B07C999006EEA2671DE7124AB
:107DB000885B3F00A332B14D5F8636BBB7B91D6B00
:107DC000B92FAB0E9B336D260E9565836E03B65CA3
:107DD000DD30836BC572C6415CE5CBE7E29B4D5E4F
:107DE000C6C5D4C4CDB02A871350B825637D663785
:107DF000AECB337BEBCB3307E176E94302883DA77B
:107E0000777784B784D2F84E46D8CA7A35CDB95937
:107E1000DF7FC70C4CEF399FFC61E185A3E6356637
:107E2000321ABC3A01027B50377240C0ADD61734CB
:107E3000F013C9A2353CD172F5ECBB723D149E60C3
:107E4000A15E2860AE119621F7F1C25A6B24E7CCEF
:107E50007EDD8983F106E58DA8E67345CDFBDEDB8B
:107E60000574340DE5CD813929B38EC24255010028
:107E7000AD42AD28812FF1B852E140BEB422C9B065
:107E800062CC44B0055D2897907D38176256B9EDF5
:107E90006B16D1C72569727D299DEA7CFE70E130A1
:107EA000A243FF65B82E84FFB084BCD7EF81AB320C
:107EB000DF357E5ED8D40C8E7628DDACE30EC18A29
:107EC000F481FE25E9095B5289AC66F615C712BC40
:107ED000DA41571EE29DA14E710BB5CDBAF4B00B3D
:107EE00027DDE56E49861A507BC7707735D76E055A
:107EF0007775E6C22B76CDB38B936E7D43B4C243C8
:107F000010047C4365BE775D46A822D007F9AE39E0
:107F10001BB6BE67CFA8DFD29C55748F4B3C1F1B8E
:107F2000A182F1EA634BDB1FB6F28E5169D2CE53C8
:107F30001622E5EFDAEFEAAFD974AFD611ED9B6206
:107F40006F04EE25BA42DC085DB6AAA7B0FC292A68
:107F5000BF775AFEB3949623960F7EA8CCCF0F3CE2
:107F60004971D25E1F16F6A35B61E374802B0E117C
:107F700004161466961BAD796E61F212F0D1BF98AB
:107F8000D4EC02018E95D598BF48C4C0644DF68EDE
:107F900089631F745C98F2DF2B081EC47BA43B84AA
:107FA000D9E93EC6C363385D414BE5DD46C6FB9566
:107FB000A54BE902A9705581D61DD8F93580C92C89
:107FC0001AAA7B7D6D5473418CABA4D7DB3DE9ECE1
:107FD0005FC4688C1476B58CB67C3AD9ED3AC2D1C0
:107FE000DCBD052BEC6452F202E138F168DBE3A55D
:107FF00071E5FF4ABCAFA91D6A69DB7C0555CE1F40
:10800000CCA26E94835671A81E0901E3967458663B
:10801000979F2BF9889E47EDA8B35AA2BFF3349ED1
:1080200049BAC3BA4C033C05870DCE2B1B99538527
:108030001B0053FB41A9288012EE366C77727C013D
:10804000D71F5FE8E0D7EAAFBF3A4F9B4B393D22DD
:10805000088A56F2FA74F06B4B17ADD49F5AC0BE23
:1080600036D1E5669D8AF8DF583A6D3B7A0C60F4AC
:10807000639995B43E89E77622B5F3E29244B57FE1
:10808000D91045C92CC6A8E24A68093F267EE0BD42
:108090001C413A8E56A257DFE63DAE5751E0A3345D
:1080A000009D1702FBB77168CF391692BA410300E1
:1080B000CB6306ADC26CDFB2F24CC7026CDFFA3B99
:1080C00035988CE0E5084FB0B4A838B9B07A85810E
:1080D000F319AC807D1C7F3B8007CF6A7B7087F5EE
:1080E0007CF7D04A552B4F698F1EBA68D593BD7265
:1080F0003FB87AD90DBF06E4F27D677F1BFB57338B
:1081000024EAA68B751A5D7D0F7E86E5A3E1B2E9B0
:108110009A2CFDAFEA009BA2651F17EAA95DBB5030
:10812000AABF7C0D412E7A2A25A0E9EA93D603C87E
:10813000EC88DF1F43FDA581F6AA1B601B32D7B078
:10814000FC0EC40EBE44EB98C092C6B182404AD623
:10815000E01A59DDB55A4DE666067AD994B925E993
:1081600082726E89906384BCE190192502F54029E2
:108170000B8D35D0CA02204EF912A2A229C2241DAD
:108180004CEF17D1242C3F1C933376C18E07D2B30A
:10819000A6D80FD4BBFCB0A1897313A23D136DA068
:1081A000BD85C264691A69958795B592470883A110
:1081B000A8B5D0D6FD38EB5266E29436486804ED97
:1081C000BEC3DEF027C9AA8E3F77AC1158B0B2B457
:1081D000D66B77D907130D723BAA8BB2C33B0F0B3B
:1081E000DA06F460757882FAD820FC2BA2350D23CC
:1081F000E59F0569A8B62CFCA407BF8FD23724AF32
:10820000F422A683C72A8A5B55A011BDD86DA9CCDC
:10821000D96B3EA0D81497A67908CD391B093E71B9
:10822000DECA8EEF821B15423234FFA05C49BA4091
:10823000BBB204A3E77DB9C1D358389A0A334B01C6
:10824000C5EFD80A35895C397AFA5222FB8FB6001D
:10825000427FE41A36EA33B6AE4B6CA591D0223594
:10826000A14B87ABA3853B7A472845779BFCC5B3D9
:108270007C2CF2054F0EC08F755040D1B4B6BB3880
:10828000ACE52085A149BEF95BEC653DC0E4C15F6A
:10829000840BA31A189E46FE79D3695115D25283D6
:1082A000294274A8AF9742B06F54DFEC1A48CEAEA3
:1082B00030A064172A84718CC2D9D6056421709EBF
:1082C0007673834D07995F54CF530E004C8764E259
:1082D000E0F328A1F91B3BCDF85F3D245609C98E78
:1082E00094BFA1D0BFBF3319F301BC4209D5299275
:1082F000FA593B1F9217C8DE71552F6A9ADC33D3A7
:1083000018E02FB34FBAA0AF4690E665865B4B806E
:108310004671C28864B9CC4F0E46BDDC48A3416E9D
:108320008AB152D065DA893AD1A81D74F54E23ACD2
:108330009FDAF0C66B5F080E4AEE5A4A658598F2DE
:10834000F1A219E5846DA6384C8DC063E8B552EFF3
:1083500031BD5CA867BC9FFA94DCDE3A76288E7F3C
:10836000A353CF52CBDFB07EBB92AFB6B860BADEBC
:10837000EAD2966F0C3B5A2260846A8B7D9823A8C0
:108380008E90D7F8717174E6B56DA8CDA054A13F59
:1083900016B7ABA80564805120343C1E4F0D324007
:1083A0004093B4A8D82A769DE9A849BC4F8D259D55
:1083B00054805432D4C0C5F48A890ABD4896FD9FC2
:1083C0001C5118BC8D7EDA06381FFA072091351F24
:1083D000C3E5F28E4D333A5402815ABC9431FADA35
:1083E00058DF16FB1FEF8DAA78FE79FF28D3559B27
:1083F0003A307D10E56F7EF3846FC430D11002FCFB
:10840000AF29E4362D6D1CC343508C814B1561DEC2
:108410005549332732C8042E7306364069D57D1B73
:10842000F0EDFEC26CCAE7499E9CC89318B65C8406
:108430007E1A68202E62D6D67474C4BC3D0697940A
:1084400045EDFAAC50A361B0DFD3AB2D47AF0BE6DF
:10845000BB3CB47F7EB92B10365A44DAF6980ACF6B
:108460002428008E05BB52F901AB82BC5AF9272D96
:10847000CFD43446702422092BD1D63373AC74DCAC
:10848000A251D46CE4949404B578AF9765A6314DAD
:10849000C69DB587A8134EE5BA7CD296B20AFB6A90
:1084A000261F91621485693F64A8435DA33E89FA43
:1084B0000949588FC70119F0BB5C0DBC3396332DA9
:1084C000CAD8AEBAF434F639EC3A133F945D2BD7E0
:1084D0009CB01230C53E4B608D620873FBEC8DFB87
:1084E000691466D5F7B56C5EDA173D3EE18C4ECF68
:1084F000FF5FBCB09266533D25DFF2E988E31F7C45
:1085000048071D832F60F3DD6E7DBE02C2C343D0DA
:108510009FAD901368F3FF3C23B41FBFE766B623FB
:108520005E555F5D7EDE2D03F9ECE1E9F356B8841C
:10853000E52FBFA064C043DF15450E07A88F1229A1
:108540003248B6B95AF218585ECC90184D8E20BFFA
:10855000698D0D8CA380C271A6F63EEEB2C2651A7B
:108560009A0BA4958A88B06F8ED8D2BC447A582DC5
:10857000A63AEF58CFF2A4AA171E69BB6621C01B0A
:108580009DEA54FE102BA1926293237177DAD71ED5
:10859000722114467FDA1B3709FB3E45C067D6259A
:1085A000673B3B5F1CEAC35ED4A899D8EE22A50EB8
:1085B000361AE3E5F3FF77D70031DC5896BE7F86A5
:1085C00099E2941ABD41C64F52A802516CD31EB213
:1085D000E25E7A64D29D586C212F4A20154B51D708
:1085E0000A83A4DD7C5576CA7348FCE7862424CA36
:1085F000C45D877C46644D63C8C3C7200D83731375
:1086000047FF14B3833E2501CB6D1E52CCD324C645
:10861000AC028FEAE009195316886AC3BFFA0CA8A6
:10862000B3D949C43DF8BE8B0AD9F62CAE9535E4D2
:1086300076B82D097D1CCA51DE062AC3B44E0CBB88
:1086400060E849E156798AF36786D42F249494141C
:1086500042A3172A96242B7F4E03E4836DD6330260
:108660006432C640115BECBA1822DCD73742E120F5
:108670009B671F6A41D3EE94DBBD5D82FA5ED4C670
:108680005487C1F034F73ECE340B097583B812E637
:108690001705B4B35EB6628D8640069BF367A0559E
:1086A0000F7386C3CF28581754BDD9248FB2945A5C
:1086B000F68E5BC8B8B2066D1009A0A3717EABA997
:1086C000E56463974587AC3B032FF887A1234C945F
:1086D000CC6C3E8849E49101D9F20B6DCA2C6E9C9A
:1086E000097AA6F683463422440F401F93B2E582EE
:1086F000D5EAC5513CA067191466EE021C73AC396B
:108700009DC7ADB85B26B5FF2FC8B5E78A9E9927F0
:108710001D143A287DEF452D6804430A3189CE04A3
:108720006996FE2D13544AF70C9107E0D124527933
:10873000A16BD687B31F55AD1707325141A4ADC207
:1087400033B0F9384A3B6E68D8EC250B477BDFCC59
:108750006FFADE096832B95B39995866C770F3D38E
:108760002A6E2505FE8C45A0853951B679813A24BB
:108770000BD08DEB830CAC00115857090F5150B63C
:10878000DC28496312B3336413CEE1EB0D42E4F00D
:1087900029F85E8101D504A75BB4B70D4D9EE0D3E7
:1087A00016D0071A7463700805110120D5E91CE67C
:1087B000E45B73D5F1A8ED96B77CDD0F0209EBE41D
:1087C000DDEFA8DC94142478F9AA5E1A1D759E4684
:1087D0003692F432881964D7F118EDF6246F5F4EA3
:1087E00037DF2330280B98E893D7DC473AAB23E3F5
:1087F000F1FE3CF68742A0660304050A08060BFF5B
:108800000209070D010C00FF202020205F5F7C0083
:108810004D454D4F525920434C454152002C00616B
:108820000044697370206F66660D0A005553455207
:10883000004600424547494E0052414400442E4DF7
:1088400059005052474D0055534552202020006694
:1088500020200067202000424547494E202020204C
:10886000200052414420202000442E4D5920202039
:10887000004320202000081C242C4448586C74031A
:108880000000000100000005000000FFFFFFFF4D99
:10889000000000FFFFFFFF0F000000F401000004D4
:1088A0000103010201010411040F04170416011849
:1088B000010000478800004F8800005388000057DF
:1088C0008800004E5700006288000069880000712F
:1088D000880000428800000502050804080B08040F
:1088E0000405010504090809040608070206020434
:1088F00002060106040701030803040C080D020C1C
:108900000203020C010C040D010D080D04080208FD
:108910000807080202070408010804090209010AFD
:10892000080B020A0201080A010A040B01020802EC
:108930000410081102100211081001100411011294
:108940000212011302130812080F08120413011374
:10895000041402140115021508140817081404154C
:108960000115041702170119081A02190216021933
:108970000119041A01160816041B021B081A08180C
:10898000021A041B011B04180818040B04202020E1
:108990002020202020202000000000030000002CC8
:1089A000880000318800004E570000338800004ED8
:1089B000570000398800003D880000976900004298
:0389C0008800002C
:00000001FF
